:020000040001F9
:10C00000184E0020C1C30100C9C30100CBC3010009
:10C01000CDC30100CFC30100D1C301000000000067
:10C02000000000000000000000000000D3C3010079
:10C03000D5C3010000000000D7C30100D9C301002F
:10C0400031C60100DBC30100CDC80100DBC3010024
:10C05000DBC30100000000008DC5010000000000EE
:10C06000DBC30100DBC30100DBC30100DBC3010054
:10C07000DBC30100DBC30100DBC30100DBC3010044
:10C08000DBC3010081C60100DBC30100DBC301008B
:10C09000DBC30100DBC30100F1C60100DBC301000B
:10C0A000DBC30100DBC30100DBC3010000000000B3
:10C0B0000000000000000000000000000000000080
:10C0C0000000000000000000000000000000000070
:10C0D000000000000000000000000000DBC30100C1
:10C0E0000000000000000000000000000000000050
:10C0F0000000000000000000000000000000000040
:10C10000000000000000000000000000000000002F
:10C11000000000000000000000000000000000001F
:10C12000000000000000000000000000000000000F
:10C1300000000000000000000000000000000000FF
:10C1400000000000000000000000000000000000EF
:10C1500000000000000000000000000000000000DF
:10C1600000000000000000000000000000000000CF
:10C1700000000000000000000000000000000000BF
:10C1800000000000000000000000000000000000AF
:10C19000000000000000000000000000000000009F
:10C1A000000000000000000000000000000000008F
:10C1B000000000000000000000000000000000007F
:10C1C000000000000000000000000000000000006F
:10C1D000000000000000000000000000000000005F
:10C1E000000000000000000000000000000000004F
:10C1F000000000000000000000000000000000003F
:10C20000DFF80CD000F084F900480047A1E90100F4
:10C21000184E002030B450E8012F93B2C489234453
:10C220008489A34228BF1B1B0489A34202BFBFF31A
:10C230002F8F002007E0C3EA020340E80134002CFE
:10C24000E9D14FF001000A6030BC704750E8012F7F
:10C25000C2EA024240E801210029F7D1704730B418
:10C2600050E8022F1FFAA2F3C488A34202BFBFF313
:10C270002F8F00200DE0C48923448489A34228BF66
:10C280001B1BC2EA034340E80234002CE8D14FF004
:10C2900001000A6030BC704750E8022FC2EA224217
:10C2A00040E802210029F7D17047034653E8022FE6
:10C2B000D988B2EB324F4FF0000017BF92B241EA7B
:10C2C000014142EA014104E05A68B2EB324F08BF33
:10C2D000012043E80212002AE8D1704730B4044636
:10C2E00054E8000F0D4644E80053002BF8D11560C8
:10C2F00030BC704730B4044654E8000F40EA0105F2
:10C3000044E80053002BF7D1156030BC704730B4BF
:10C31000044654E8000F00EA010544E80053002BEE
:10C32000F7D1156030BC704730B4044654E8000FB4
:10C3300080EA010544E80053002BF7D1156030BCBA
:10C34000704730B4044654E8000F00EB010544E8A0
:10C350000053002BF7D1156030BC704730B4044651
:10C3600054E8000FA0EB010544E80053002BF7D17F
:10C37000156030BC704770B404464FF0000054E8BC
:10C38000006F0D68AE4207BF44E80023012044E877
:10C3900000630E60002B1CBF0020F0E770BC7047EC
:10C3A00030B4044654E8000F88422CBF451A0546B5
:10C3B00044E80053002BF5D1156030BC70470000F5
:10C3C0000648804706480047FEE7FEE7FEE7FEE72F
:10C3D000FEE7FEE7FEE7FEE7FEE7FEE7F5C6010043
:10C3E00001C201002DE9F05F0546002092469B4600
:10C3F00088460646814640241BE02846414647467B
:10C40000224600F074F853465A46C01A914110D3A0
:10C4100011461846224600F016F82D1A67EB01085F
:10C420004F4622460120002100F00DF817EB0009CD
:10C430004E41201EA4F10104DFDC484631462A4665
:10C440004346BDE8F09F202A04DB203A00FA02F1BF
:10C45000002070479140C2F1200320FA03F31943F2
:10C460009040704700487047DC27020040EA010313
:10C470009B0703D009E008C9121F08C0042AFAD29A
:10C4800003E011F8013B00F8013B521EF9D270475E
:10C49000D2B201E000F8012B491EFBD27047002206
:10C4A000F6E710B513460A4604461946FFF7F0FFB3
:10C4B000204610BD421C10F8011B0029FBD1801A38
:10C4C000704730B504460020034600E05B1C9342F1
:10C4D00003D2E05CCD5C401BF8D030BD034611F8C0
:10C4E000012B00F8012B002AF9D118467047202AA9
:10C4F00004DB203A21FA02F00021704721FA02F30E
:10C50000D040C2F120029140084319467047000014
:10C51000064C074D06E0E06840F0010394E8070090
:10C5200098471034AC42F6D3FFF76EFE0C30020091
:10C530002C30020070B58C1810F8015B15F0070361
:10C5400001D110F8013B2A1106D110F8012B03E0AC
:10C5500010F8016B01F8016B5B1EF9D12B0705D4B4
:10C560000023521E0DD401F8013BFAE710F8013BFD
:10C57000CB1A921C03E013F8015B01F8015B521E19
:10C58000F9D5A142D8D3002070BD00002DE9F843B1
:10C590000025DFF894804FF4807601242F46009523
:10C5A000304603F045F938B1D8F80403204203D0EF
:10C5B000304603F033F92543361D64007F1CB6B2C4
:10C5C000082FEDD34FF4BE74204603F031F948B183
:10C5D000204603F023F945F000456A46012100207A
:10C5E00003F0DAF815F0FF0F16D0012600242E42D2
:10C5F0000ED008EB8401D1F81005D1F81015C0F366
:10C6000004200A4AC1F3014152F8242002B19047A4
:10C610007600641C082CEAD3002D02DA684604F088
:10C620005BFEBDE8F8830000006000405C34002041
:10C6300070B54FF48076304602F08AFE0F4DB40597
:10C6400040B1304602F08BFE0120C4F8080329688F
:10C65000002088474FF48276304602F079FE0028A9
:10C660000AD0304602F07BFE0220C4F80803296895
:10C67000BDE870400120084770BD0000E42D002097
:10C6800002490248091F096800680847542E002023
:10C6900000F022B970B50E46144900EB400001EBE2
:10C6A000C0051446E86A183520B101280FD00228C9
:10C6B00005D113E0284600F043F9A04201D200243E
:10C6C00011E022463146284600F072F90BE0284678
:10C6D00000F036F9A042F4D20446F2E7314628468B
:10C6E00000F039F90446204670BD0000903B002060
:10C6F00003F0C8BEF0B54FF08051684FD1F830015B
:10C70000674E421C09D0D1F834410346012500226E
:10C710000D2B07D0102B05D00FE032783B78C2F3F9
:10C720000314F3E70CB1012C07D14FF08043C3F899
:10C730000C21C3F810215B4B1A60431C07D0D1F8C1
:10C74000344103460D2B07D0102B05D05DE0347823
:10C750003B78C4F30314F5E70CB1012C55D1524BCF
:10C760001B68524C2360504B1B1D1B68241D23600B
:10C770004D4B08331B68241D23604B4B0C331B6847
:10C78000241D2360484B10331B68241D2360464B37
:10C7900014331B68241D2360434B18331B68434C20
:10C7A00020342360404B1C331B68241D23603E4B08
:10C7B00020331B68241D23603B4B24331B68241D3E
:10C7C0002360394B28331B68241D2360364B2C33E0
:10C7D0001B68241D2360344B30331B68334C4034BA
:10C7E0002360314B34331B68241D23602E4B3833B8
:10C7F0001B68241D23602C4B3C331B68241D2360C5
:10C80000294B40331B68241D2360431C06D0D1F8FC
:10C8100034110D2807D0102805D00EE03178387873
:10C82000C1F30311F5E709B1012906D120480168D8
:10C83000C90702D06FF0010101604FF01021D1F85B
:10C840000002002803DBD1F80402002821DA194C89
:10C85000256019480368002BFCD01223C1F8003270
:10C860000568002DFCD0C1F8043201680029FCD015
:10C87000226001680029FCD0BFF34F8F0F48016888
:10C880000F4A01F4E06111430160BFF34F8F00BF15
:10C89000FDE70D490B480860F0BD0000E00F00F017
:10C8A000E80F00F0380500400404001020C50040E7
:10C8B0000004004004E5014000E401400CED00E00C
:10C8C0000400FA050090D003CC2E00200148006837
:10C8D00000470000EC2D002010B5124C0220206112
:10C8E000606111A0A06104F17800E0614FF4007074
:10C8F00020620020A06260620BA1A164E06204F5E6
:10C900001E71E1641021A065C4E91410E06509A15D
:10C91000E01DFFF7E3FD08A12046FFF7DFFD202023
:10C92000A07110BD903B00205465726D696E616C02
:10C930000000000052545400534547474552000040
:10C940000269C1688A4203D88068401A104400E036
:10C95000501A401E70472DE9F047C46817468946B3
:10C9600006464FF000083069A04201D9051B02E0DD
:10C97000B168201A0D1AB0686D1E001BA84200D8BD
:10C980000546BD4200D33D4670682A4620444946CC
:10C99000FFF76CFDB0687F1B2C44A844A944A0425B
:10C9A00000D10024F460002FDDD14046BDE8F087BF
:10C9B0002DE9F04104468846D4E90207C51BE16829
:10C9C000606816460844B54206D94146FFF74EFD59
:10C9D000B819E060BDE8F0812A464146FFF746FD00
:10C9E000761B08EB050132466068FFF73FFDE66005
:10C9F000F0E70000014A024900F026B82BE50100EB
:10CA0000642E002002E008C8121F08C1002AFAD1D3
:10CA100070477047002001E001C1121F002AFBD1BE
:10CA2000704700000121202803DA814005480140B9
:10CA300003E0402802DA2038814009B10120704724
:10CA400000207047FC06FFBD2DE9F04116460F4659
:10CA50000446002503E03946B047641C6D1C20786D
:10CA60000028F8D12846BDE8F08110B50122022146
:10CA7000002000F08FFF08B1072810D10722022103
:10CA8000012000F087FF08B1072808D100210A2201
:10CA9000084600F07FFF08B1072800D1002010BD34
:10CAA000022000F093BE000070B50024064D06E0A1
:10CAB0006868012110F8340003F0FAFD641C28783E
:10CAC0008442F5D3002070BDF82D0020F8B516463D
:10CAD0000C4605460A2A01D20720F8BD03F0E2FE03
:10CAE00018B903F0A5FE0028F7D1134F1021134801
:10CAF0007D603C70BE60FFF7D2FC0020C7E90400F7
:10CB00000F4E0DE005EBC4003168009181788DF87F
:10CB1000011000780B4A694603F01AFE0028DCD1A8
:10CB2000641EE4B2EED2BDE8F84005480021064A92
:10CB3000001D00F087B80000F82D002028350020E7
:10CB4000D0240200A5E6010081DF010072B603F0E7
:10CB500009F900BF02F03CFF0028FBD1114812493F
:10CB6000401AC408012000EB044010A103F04CF867
:10CB700011480068C00700D000BE022000EB04404E
:10CB80000EA103F041F8BFF34F8F0B48E438016862
:10CB90000E4A01F4E06111430160BFF34F8F00BF03
:10CBA000FDE70000B43002003C30020046617461D1
:10CBB0006C206572726F7200F0ED00E0537973744F
:10CBC000656D207265736574000000000400FA054D
:10CBD0000EB500210091CDE901106A4644F2010032
:10CBE000FFF7B4FF0EBD10B58268C368934203D04F
:10CBF00001F088FC002010BD052010BD29B112B144
:10CC0000531E134203D0092070470E207047016065
:10CC1000838000218160C1600846704710B582683A
:10CC2000C3689A1A83889A4203D801F075FC0020E1
:10CC300010BD042010BD0000014801F0E0BA000062
:10CC4000182E00203AB100680129426100D000216D
:10CC500001610020704707207047000038B5114877
:10CC600008235822416800910F49006801F0AAFF8B
:10CC7000002815D10D4A69460D4801F0C5FA040097
:10CC80000ED101210A4801F03AFB0123094A194655
:10CC9000074801F08CFA064901200839087020463F
:10CCA00038BD0000D8240200483500204517020096
:10CCB000182E0020FFFF7F0070B50446007F0D4650
:10CCC00008B1002070BDA26101F0D2FC401941F111
:10CCD0000001C4E90201206900B125612146BDE8D7
:10CCE0007040002005F070B8014600200877012050
:10CCF00005F06AB870B50A4E01460A48B578FFF7E4
:10CD000072FF04464DB10020B070711C0122C81D95
:10CD100002F09CFB08B1FFF75BFF204670BD0000EE
:10CD2000342E0020A0350020F0B5244E89B01F46D7
:10CD30000D00044672603FD0A888296882B220485E
:10CD4000FFF75CFF002835D1A889A96882B21C488A
:10CD50001030FFF753FF00282CD1202219496846D4
:10CD6000FFF784FB60690690207C00B101208DF8FC
:10CD700014008DF81C70607C00B10E208DF8150039
:10CD8000E0680290A06803902068019060680090BD
:10CD90000A480D4A6946083002F024FB002809D1F0
:10CDA000B0702068401C05D004490122491CC81DF0
:10CDB00002F04CFB09B0F0BD0720FBE7342E002049
:10CDC000A0350020EC240200591F020010B50146D6
:10CDD0001048FFF723FF040019D10F480F4A0178CC
:10CDE000515C19B1001D03F0EFFF02E00C3003F0BD
:10CDF000C5FE60B9084907480839FFF7F4FE30B9A5
:10CE0000054901220839044802F030FB0446204657
:10CE100010BD0000B03500203C2E0020D82D002091
:10CE200030B5EFF3108172B60D4A9468012324B136
:10CE30000370002900D162B630BD93604FF0E0234B
:10CE4000D3F88051074C25401560C3F88041D3F8D2
:10CE5000844154605A17C3F8842100220270E8E725
:10CE6000C0350020FC06FFBD0B498A68002A11D09E
:10CE700000280FD1EFF3108072B60B684FF0E0225C
:10CE8000C2F800314B68C2F8043100228A600028E1
:10CE900000D162B670470000C03500202DE9F04196
:10CEA000064608680C46411C4FF0A0474FF00105AC
:10CEB00006D005FA00F1C7F80815206802F046FC14
:10CEC0006068411C02D0002102F02EFC3168A0698C
:10CED000C1F82405607D227D31681043C1F86C05DE
:10CEE000D4E900123068C0F81425C0F80C15207D74
:10CEF000012815D1A068411C02D0002102F014FCC9
:10CF0000E068411C05D08540C7F80855E06802F08C
:10CF10001DFCD4E902123068C0F80825C0F81015CD
:10CF2000BDE8F0812DE9F041064608680C46411C39
:10CF30004FF0A0474FF0010506D005FA00F1C7F801
:10CF40000815206802F00CFC6068411C02D000212A
:10CF500002F0F3FB3168A069C1F82405607D217DF2
:10CF600032680843C2F86C05D4E900123068C0F892
:10CF70000C15C0F81425207D012815D1A068411C8E
:10CF800002D0002102F0D9FBE068411C05D08540A9
:10CF9000C7F80855E06802F0E3FBD4E902123068F4
:10CFA000C0F80825C0F81015BDE8F08170B5E0B1F3
:10CFB000DAB1002402E0045D2C44A4B2651C8D4269
:10CFC00006D21688A642F6D8061976789E42F2D185
:10CFD0008C420AD2A31C005D9BB200B1401E00042B
:10CFE000000C02D01C188C4201D9002070BD1380A7
:10CFF00070BD2DE9F0418AB006460020ADF814005E
:10D000001346102088468DF804000D4606AA01A993
:10D01000184665DFA6B398BB9DF80400022804D02B
:10D02000042807D0102839D10DE003208DF8100016
:10D03000022003E005208DF8100004208DF8110077
:10D04000002404AF0FE007208DF810000620F5E75C
:10D050003B5D05AA41463046FFF7A8FF641CE4B2D9
:10D060000546022C04D2BDF814000028F0D003E0DD
:10D07000BDF81400002812D080B2064400240BE052
:10D080000CE030199DF8042006A9FFF71AFA48B100
:10D090009DF80400204484B2AC42F2D300200AB0D0
:10D0A000BDE8F0810120FAE770B540B10C4D297858
:10D0B00039B1044604F0ACFA28B1002070BD0E204E
:10D0C00070BD082070BDE868062807D205492268AF
:10D0D00001EB8001401C0A60E860EEE7042070BDAF
:10D0E000C82D00203034002010B558B103684BB172
:10D0F00042683AB1044900200124C8600C70C1E9BB
:10D10000013210BD0E2010BDC82D0020002827D0F0
:10D11000002925D0134A1278002A21D00A46018816
:10D12000112911D0302907D0322909D0332917D13C
:10D13000011D104603F038BF011D104603F0F8BF73
:10D14000011D104603F050BE8088B2F8CA12884212
:10D1500006D1002082F8C8024FF6FF70A2F8CA027A
:10D1600070470000C82D002048B1084A137843B129
:10D17000D26832B190F8C8222AB1112070470E202F
:10D1800070470820704700F0B9BF0000C82D00208C
:10D1900038B50288011D04461F2A47D016DC102A24
:10D1A0001ED02B482B4BC01AC008032303EB0040B2
:10D1B000112A2DD0132A33D01B2A44D109790229F0
:10D1C00041D1BDE8384024A102F01EBD212A31D052
:10D1D0003B2A39D0562A36D1A088132177DF11E0B7
:10D1E000A1880022244800F001F908B1FFF7F0FC03
:10D1F000072000F0F1FB08B1FFF7EAFCA1881F4807
:10D20000FFF7B2FF00281ED0BDE83840FFF7E0BCB2
:10D210000B790A8801B01AA1BDE8304002F0FFBCCA
:10D220000023A0881A46852180DFEBE731F8040B44
:10D2300076DFE7E700200090A08869468DDF0028B0
:10D2400001D0FFF7C5FC38BDA088132177DFD9E7EF
:10D25000B43002003C300200436F6E6E6563746947
:10D260006F6E20526571756573742074696D6564A5
:10D27000206F75742E000000C4310020B4270020F8
:10D28000446973636F6E6E65637465642E20636FAB
:10D290006E6E5F68616E646C653A20307825782C1C
:10D2A00020726561736F6E3A203078257800000037
:10D2B00010B51A4C0188606810290ED011292BD1A5
:10D2C000401E606028D1FFF7D0FB002824D02168E1
:10D2D000002921D0BDE810400847D0B90021012223
:10D2E000084600F057FB08B107280FD1072202219A
:10D2F000012000F04FFB08B1072807D104220221CA
:10D30000002000F047FB20B1072802D0216801B1BE
:10D3100088476068401C606010BD0000C02D002080
:10D3200070B506461A481B4A0D46801AC00809788F
:10D33000032202EB004459B1012922D0022926D14F
:10D34000204615A102F060FCBDE8704004F050BB1F
:10D35000204615A102F058FC698805F10E023046FE
:10D3600000F044F808B1FFF733FC304600F04AF90A
:10D3700008B1FFF72DFC2046BDE870400FA102F078
:10D3800043BCA989A868BDE8704000F071B970BDC0
:10D39000B43002003C300200446973636F6E6E6506
:10D3A000637465642E000000446973636F76657270
:10D3B0007920636F6D706C6574652E00436F6E6EBF
:10D3C000656374656420746F2064657669636520A5
:10D3D00077697468204E6F726469632055415254B6
:10D3E00020536572766963652E00000050B141805C
:10D3F0002AB15388C3801388838092880281406950
:10D4000001F032BD0E20704730B5144B0D460400BC
:10D410000FCB85B08DE80F001ED0EDB1A868D8B154
:10D420002146684662DF002814D120788DF812006A
:10D430000120ADF810004FF6FF7060802868E060B2
:10D44000686820610020A0802081A868606104A82D
:10D45000FFF72AFE05B030BD0E20FBE7B424020022
:10D4600030B5024685B008002DD0002A2BD0418867
:10D470004FF6FF74A14226D09388994223D1158894
:10D48000112D14D0392D1ED1818800291BD053892C
:10D490008B4218D1C168002915D001218DF80010E8
:10D4A00002F110010291D189ADF80C1008E08B4215
:10D4B00009D1C168002906D002218DF800104480EE
:10D4C000C2686946904705B030BD30B585B00C469E
:10D4D000054614216846FEF7E2FF207804F10E01AC
:10D4E000002830D1A08801282DD1A0792A78904237
:10D4F00029D1002217E002EBC20031F81030022BD4
:10D5000002D0032B0ED105E001EB40000089ADF8FD
:10D51000120007E001EB40000389ADF80E304089AE
:10D52000ADF81000521C207A9042E4D8E868002838
:10D5300009D06088ADF8020000208DF80000EA688C
:10D5400069462846904705B030BD000070B588B0E8
:10D5500015460E46040012D020216846FEF79FFFB4
:10D5600019481A49401AC008022101EB0040F42D65
:10D5700007D917A102F048FB072008B070BD0E20A4
:10D58000FBE76288A2F57F43FF3B18D0154ACDE93F
:10D59000022401208DF800002289ADF812208DF8B8
:10D5A0001010ADF816500022ADF8142006968DF834
:10D5B000110062886946606901F08EFCDDE70AA10E
:10D5C00002F022FB0820D8E75C3002003C30020069
:10D5D000436F6E74656E7420746F6F206C6F6E672E
:10D5E0002E00000039E50100436F6E6E65637469BB
:10D5F0006F6E2068616E646C6520696E76616C691F
:10D60000642E000010B58AB058B34188A1F57F425E
:10D61000FF3A28D0C18831B3044620216846FEF77E
:10D620003EFF01218DF8201000208DF821000F4AC7
:10D63000CDE902248DF80010E288ADF81220022214
:10D64000ADF81620ADF814008DF8101008A88DF86C
:10D650001110069062886946606901F03DFC0AB0CD
:10D6600010BD0E20FBE70820F9E7000039E50100B6
:10D670002DE9F0410E4605461C481D490024401A7C
:10D68000C008012101EB00480FE0285DFFF79EFB79
:10D69000070009D0112FF8D04046224615A102F00C
:10D6A000B7FA3846FFF794FA641CB442EDD3A819D0
:10D6B00010F8010C0D2804D10A20FFF787FB112870
:10D6C000FAD0324629461548FFF740FF04000BD038
:10D6D000112CF6D04046224611A102F099FA2046BC
:10D6E000BDE8F041FFF774BABDE8F081B430020044
:10D6F0003C3002006170705F756172745F707574A8
:10D70000206661696C656420666F7220696E64656D
:10D7100078203078253034782E000000C431002085
:10D720004661696C65642073656E64696E67204E3E
:10D730005553206D6573736167652E204572726F56
:10D740007220307825782E20000000000149085C06
:10D7500070470000E02302000649095C4FF0A0403A
:10D76000D0F81005C84010F0010000D0012080F072
:10D7700001007047E02302002DE9FC410646C00786
:10D780004FF000050ED0104F00240122385D0095A7
:10D7900000231146019501F07FFF641C042CF4D393
:10D7A00000F046F8B0070DD5074E0024361D0022C4
:10D7B000305D032300951146019501F06DFF641C57
:10D7C000042CF4D3BDE8FC81DC23020007490B5C88
:10D7D0004FF0A041D1F804250120984020EA02032F
:10D7E000C1F808351040C1F80C057047DC23020071
:10D7F0000249085C012102F005B80000DC230200A8
:10D800000249085C002101F0FDBF0000DC2302009A
:10D810000649095C4FF0A040D0F80405C84010F05C
:10D82000010000D0012080F001007047DC230200DD
:10D8300010B500242046FFF7DBFF641C042CF9D34D
:10D8400010BD10B500242046FFF7DAFF641C042C3D
:10D85000F9D310BD10B50246064B4FF0FF30002142
:10D860005C5C944201D1084610BD491C0429F7D3E1
:10D8700010BD0000E023020070B50C4E0C004FF00C
:10D88000000530600BD0012000F06AF808B10220DA
:10D8900004E0002000F064F800B10B2020707068F4
:10D8A00010B9FFF7E2F80546284670BDC02D0020EC
:10D8B00010B5002000F0CAF908B1062806D10120F1
:10D8C00000F0C4F908B1062800D1002010BD000006
:10D8D0002DE9F0470D468146FFF7BCFF04460428BA
:10D8E00036D2DFF874801B481C4EA8F10C0725B314
:10D8F000012D0ED0022D2BD104EB4400304445788D
:10D90000002D25D0B968002922D02846BDE8F0476F
:10D91000084704EB4401755C0E44717849B10E4A26
:10D920004FF48041093A8068FFF7C6F908B987F8D3
:10D930000390B17808F80410E2E78068FFF7D4F9A3
:10D9400004EB4401314418F804008D78A842D7D084
:10D95000BDE8F087E4230200BC2D00200034002045
:10D96000042801D2FFF7F8BE00207047042804D035
:10D970000A280CD1002002F0F1BA05481321408892
:10D9800077DF082803D0002801D0FFF721B97047BE
:10D99000C431002070B50023042810D20D4D00EBD7
:10D9A0004004012A02D101290CD00022094E00EBCB
:10D9B0004000304461B1012906D0022906D0072376
:10D9C000184670BD0E30C2B22A55F9E74270F7E72B
:10D9D0008270F5E700340020044A014600201279E5
:10D9E000D20702D0084600F04DB87047B02D002095
:10D9F00070B506461E480024C0E90161B00720D575
:10DA00000025012211462846FFF7C4FF6D1C04467D
:10DA1000042D02D2002CF4D013E094B940F233323A
:10DA200004211448FFF752F804000AD1FFF73CF82C
:10DA3000040006D10F48104A0021001FFFF702F929
:10DA40000446F00712D00120FFF796FE74B909488A
:10DA50000A4A00210C38FFF7F5F8040006D1054802
:10DA6000074A01210838FFF7EDF80446204670BD4B
:10DA7000B02D0020F023020059DD0100D9E801009B
:10DA8000A1CA01002DE9F05F6E4C054600266078C2
:10DA9000B34618B184F801B000F006FF6A4F4FF4A6
:10DAA0007A694FF4C87A4FF00108182D69D2DFE87F
:10DAB00005F00C1313384754696E727B727BC58472
:10DAC00084848484B3B6B9BCC5C500F0EDFE386863
:10DAD000FFF70AF906465CE00020FFF799FE0028F0
:10DAE0004FF0000008D0FFF783FE022D02D14FF463
:10DAF000E16008E0484606E0FFF782FE022D01D112
:10DB0000C82000E05046410CC0034FF47A728018E0
:10DB100041F10001257052000023FEF763FC01462D
:10DB20002AE00020FFF774FE00284FF0000004D028
:10DB3000FFF75EFE4FF44870E5E7FFF761FEDFE7B1
:10DB40000020FFF765FE00284FF0000002D0FFF72D
:10DB50004FFECFE7FFF754FED4E70020FFF758FE53
:10DB600000284FF0000002D0FFF742FE01E0FFF76F
:10DB700047FE257040F6CD4100223868FFF79CF83B
:10DB8000064646E00020FFF721FE257008E0002051
:10DB900051E025703DE084F801800120FFF716FE7A
:10DBA000002240F26661E8E784F801800120FFF777
:10DBB0000DFE00224FF40051DFE77868FFF794F87C
:10DBC0000646D5F1110000D02EB10220FFF710FE5D
:10DBD00084F802B01DE0012816D980B2C82148435C
:10DBE000C117C90341EA5041C0034FF47A7280184B
:10DBF00041F1000152000023FEF7F4FB0146002230
:10DC00007868FFF759F806460220FFF7F9FD84F817
:10DC100002803046BDE8F09F00F046FEB9E700F014
:10DC200043FEB4E700F040FE04E000F03DFE0020BB
:10DC3000FFF7E6FD0120FFF7E3FDAAE7FFF701FE8E
:10DC4000A7E70000B02D0020E4230200012104F02A
:10DC50008FBB00002DE9F84F0546861C00208DF88B
:10DC6000000091460F464FF0010A6846FFF7D8F8CA
:10DC70001B4C04F21C4860683860D4E90101194F5C
:10DC8000401A3968081A0EE00121404600F0DFFF13
:10DC900000F034FE0146404600F0D9FFD4E901010E
:10DCA000401A3968081A401C8642EDD8B9F1000FB5
:10DCB00003D0052065F3891002E0062065F39F502C
:10DCC00061683A68114004EB8101C86060683044C3
:10DCD00060609DF80000FFF7C7F85046BDE8F88F78
:10DCE00070370020742E002070B50D4604460A29B6
:10DCF00002D10D21FFF7F8FFA0682268411CA16046
:10DD00001554D4E90101814204D32046BDE8704096
:10DD100001F0C9BB70BD00000448816840688142C1
:10DD200001D10120704700207047000070370020AB
:10DD3000034630B5074800210478426806E000BF7A
:10DD400002EBC10005789D4203D0491CA142F7DBDC
:10DD5000002030BDF82D002000780221FFF7B8BD6B
:10DD600005494FF0FF32082841F8202002D308442B
:10DD700080F84820704700005C340020F0B54FF078
:10DD8000FF3512B10023082601E008230C260C4CB5
:10DD900005E000BF54F823707F1C04D05B1CB34225
:10DDA000F8D32846F0BD26185DB286F8305044F806
:10DDB0002310002AF5D1E11881F84800F1E70000AE
:10DDC0005C3400200249084490F93000704700009C
:10DDD0005C34002030B589B00D46044620216846E9
:10DDE000FEF75DFB94F8C602002300EB8001C1EB57
:10DDF000801094F8C51204EB400041B1491EC9B22D
:10DE000001EBC10100EB4101498A491C00E0C188D6
:10DE1000008961F30F0360F31F4303208DF80000B6
:10DE20000548CDE90204054804932A4669468068FE
:10DE300001F052F809B030BDADE00100C82D00205E
:10DE400070B5084C050009D010342168002907D0AE
:10DE500008682060496828468847F6E70834F4E7F0
:10DE600070BD000048340020054A012120B101287E
:10DE700005D19170FFF7E4BF51700020FAE77047B9
:10DE80004834002010B5D0E90234D1E90220D11A7B
:10DE9000A04101D3012010BD002010BD10B50246E5
:10DEA0000020138806E0546834F810408C4203D0F8
:10DEB000401C80B28342F6D810BD000001460148E4
:10DEC000FFF703BBC43100202DE9F04389B00F46B2
:10DED0000546914620216846FEF7E1FA95F8C6020C
:10DEE00095F8C54200EB8001C1EB801005EB4006C0
:10DEF00004EBC40006EB40013279601C0A31904209
:10DF000032D108AB0022284600F09CFC78B310E028
:10DF1000401EA04201D1002004E004EBC40006EB47
:10DF200040001C308046024608AB284600F08AFCC0
:10DF300090B10020387004208DF8000008984A46FF
:10DF4000CDE903500C4802900C486946806800F007
:10DF5000C3FF09B0BDE8F08395F8C5024146401CF7
:10DF6000641C85F8C502E4B23079A042D0D8012003
:10DF700038700020EDE70000ADE00100C82D002062
:10DF800070B500240F4D10E0686800EBC4063078CF
:10DF900002F044FC7178012901D0012100E0002148
:10DFA0004140307800F034FA641C28788442EBDB7E
:10DFB000D5E90401084303D0BDE8704003F020BF59
:10DFC00070BD0000F82D002030B59FB00C4605460E
:10DFD0007C216846FEF763FAADF8024003208DF815
:10DFE0000000044801954168002901D0684688472F
:10DFF0001FB030BDC82D00202DE9F041044690F837
:10E00000C602884600EB8001C1EB801004EB40069D
:10E010001746304603F0FCFA050042D0D4F8CC0293
:10E0200006283ED204EBC0107622A0F8D272D4F8B3
:10E03000CC02314604EBC01000F53570FEF716FA3D
:10E040000026B8F1000F06D0D4F8CC0204EBC010C3
:10E0500080F8D06206E0D4F8CC12022004EBC111A3
:10E0600081F8D002D4F8CC0204EBC010C0F84C53B5
:10E07000D4F8CC020C4D401CC4F8CC02E9688842AC
:10E080000FD12746002407E007EBC41101F53470D7
:10E09000D1F84C138847641CE8688442F4D3C7F86D
:10E0A000CC62BDE8F0810000C82D0020F0B5154617
:10E0B0009FB0002281F8C822074691F8C6020C469C
:10E0C00000EB8002C2EB801001EB400003F0A0FAED
:10E0D000060009D07C2208496846FEF7C7F9ADF86A
:10E0E000025068460197B0471FB029462046BDE858
:10E0F000F040FFF769BF000010240200F0B50D46A4
:10E1000089B004464FF4BA61FEF7C9F92021684688
:10E11000FEF7C5F9154E2946B06800F0A5FE0028A7
:10E1200021D1A4F8CA52C4F8CC0284F8C70284F8FA
:10E13000C60284F8C5020E4801272A4600682060FE
:10E1400002208DF80000ADF810702068CDF81200A4
:10E150000848CDE902046946B06800F0BDFE002819
:10E1600001D184F8C87209B0F0BD0000C82D0020AC
:10E1700030340020ADE0010010B50021024800F06D
:10E1800071FD80F3100010BD8C3B00204FF48032F5
:10E190008A400168C1F848230068C0F80823704726
:10E1A0004FF4A07202EB810189B200F0A1B92DE910
:10E1B000F04105460E464FF4A07000EB860081B298
:10E1C00028684FF48034B440984622F07F47C0F866
:10E1D00008432868C0F84843286801F0AAFF286867
:10E1E00000EB8600C0F840752868C0F84443B8F1D9
:10E1F000000F02D02868C0F80443BDE8F081006831
:10E20000D0F804057047000070B54379234C44F8FA
:10E2100023204279231D03EBC202224C1579204AA8
:10E22000121BD4082DB10825022000EB04401EA1CA
:10E2300030E005680A88C5F8082590F90420897837
:10E24000002A4FEA411104DB02F1E02282F80014B7
:10E2500005E002F00F0202F1E02282F8141D90F9AD
:10E2600004100122002909DB01F01F0502FA05F55F
:10E270004909890001F1E021C1F8005141790025E7
:10E2800003EBC1010A71417943F83100032000EB2F
:10E2900004400EA101F0B8FC284670BD502E0020AD
:10E2A0009C3002003C30020052544320696E73746B
:10E2B000616E636520616C726561647920696E6965
:10E2C0007469616C697A65642E0000005254433AA7
:10E2D00020696E697469616C697A65642E0000005A
:10E2E00090F90400002809DB00F01F020121914091
:10E2F0004009800000F1E020C0F8001270470A4693
:10E30000022100F07BB84FF4827100F0F1B8006890
:10E3100001210160704700680121416070472DE9CB
:10E32000F05F07460C464FF4A07000EB84001FFA24
:10E3300080FA38684FF48036A6409B4622F07F452D
:10E34000C0F848633868C0F808633868D0F80485B6
:10E3500000EB8402D2F84095C2F8408551463868F7
:10E3600001F0E7FEA9EB080020F07F40012806D16C
:10E37000102002F095F95146386801F0DAFE38684D
:10E38000D0F80485C0F84463A5EB080121F07F4173
:10E390003868012900EB840010D0C0F84055386877
:10E3A000D0F804156FF07F4C6A1A521E22F07F429B
:10E3B000ACEB0B03934217D362B118E06D1CC0F8AD
:10E3C0004055102002F06CF93868D0F8040540453B
:10E3D0000AD10CE000EB84006D1CC0F84055386891
:10E3E000D0F80405884202D00D20BDE8F09F01223C
:10E3F0003146384600F002F80020F6E70368C3F81B
:10E400004413002A02D00068C0F8041370470000CB
:10E410002DE9F84F0E463449804601EB5001C00704
:10E42000097801D00F0901E001F00F074FF0000952
:10E43000424601204946FEF706F8DFF8B0A0044640
:10E440000D46052F4ED2DFE807F003161B282C00DF
:10E45000002E47D00121404603F0ECFB8DF80090E0
:10E460006846FEF7DDFC5046D0E904120C43154324
:10E47000CAE9044532E00EB1022114E0002112E0A5
:10E480004EB10321404603F0D5FB4046BDE8F84FAE
:10E49000012103F05DBF012105E0002E22D10421FE
:10E4A00001E02EB103214046BDE8F84F03F0C2BBA6
:10E4B0000021404603F0BEFB0021404603F048FF28
:10E4C0008DF800906846FEF7ABFC5046E243D0E979
:10E4D00004341A4024EA0501CAE904219DF8000029
:10E4E000FEF7C2FCBDE8F88F28350020F82D00208B
:10E4F00010B5006842581AB101F01BFE012010BD92
:10E50000002010BD826883881A4003689A5C0A70F4
:10E510008168491C81607047C26883881A4003681B
:10E520009954C168491CC160704710B50446C0B217
:10E53000FEF74CFC204610BD0969002900D00847B1
:10E540007047000070B508880D46A0F52061773946
:10E5500016D10C480C49401AC108032000EB0144B5
:10E560000AA1204601F050FBA88810A1C01E82B26B
:10E570000D48134602802046BDE8704001F04FBBB5
:10E5800070BD0000B43002003C3002004154542001
:10E590004D54552065786368616E676520636F6DC3
:10E5A000706C657465642E00B0270020426C652095
:10E5B0004E5553206D61782064617461206C656EE6
:10E5C0006774682073657420746F2030782558282C
:10E5D0002564290010B50949094800F0BAFB08B1C3
:10E5E000FEF7F6FAF721064800F0A7FB002803D053
:10E5F000BDE81040FEF7ECBA10BD000045E5010093
:10E60000DC31002070B50D4601F11004C98A1029D3
:10E6100001D9092070BD01F014FC686030B1E288B6
:10E620000023A16801F073FC002070BD042070BDC0
:10E6300070B50D4601F1100489690988102901D9C6
:10E64000092070BD891C01F0FCFB686068B10023E3
:10E650000222A16801F05BFCA068E1680223028845
:10E66000686801F054FC002070BD042070BD0000FB
:10E6700010B50B48FFF7C3FD094A083AD2E9043444
:10E68000C018D2E9063244F10001C31A71EB02024C
:10E6900004D24FF08072801841F1000110BD0000DB
:10E6A000182E002010B5C0B2FFF742FB04460078D8
:10E6B00002F0B4F801466078012801D0012000E0A2
:10E6C000002090EA010F08D00449D1E90401084371
:10E6D00003D1BDE8104003F093BB10BDF82D00201E
:10E6E0002DE9FC5F0E008346DDE90C47C6F1000012
:10E6F00098469246814600D40846012503E000BFB3
:10E7000090FBFAF06D1C5045FADAA84500D9454651
:10E7100024B1002E01DB780700D5641EB80702D5AE
:10E72000B8F1000F0AD0F80708D13CB1A54205D2D4
:10E7300020215846641EFFF7D7FAF6E7002E02DACA
:10E740004E462D2102E0780703D52B215846FFF7CE
:10E75000CBFA07F0030002280BD1B8F1000F08D163
:10E760003CB1A54205D230215846641EFFF7BCFAE1
:10E77000F6E7CDE90047434652463146584603F096
:10E780008DFDBDE8FC9F000070B50D460446006895
:10E790004FF4887101F03AFF4FF49071206801F056
:10E7A00035FF4FF49271206801F030FF4FF4A271F1
:10E7B000206801F02BFF4FF4AC71206801F026FFB8
:10E7C00020681249C0F804132068690740F3073035
:10E7D000090E002804DB00F1E02080F8001405E0B9
:10E7E00000F00F0000F1E02080F8141D206840F3D5
:10E7F0000730002809DB00F01F0201219140400989
:10E80000800000F1E020C0F8001170BD100342004C
:10E81000024600201268530713D502F003000128B6
:10E8200002D002280CD105E0C2F383100B68801CD3
:10E83000184404E00223086803EB92521044086075
:10E840000120704710B509892AB1D088491C81423E
:10E8500018D1002010BD90F8C62202EB8204C4EB50
:10E86000821200EB420212899142F2D0491C1980B7
:10E8700090F8C61201EB8102C2EB811100EB41005E
:10E88000008902E01980D088401E5880012010BD08
:10E89000007DC0F3C100012803D0032801D000206F
:10E8A00070470120704700000A4810B5807860B1B9
:10E8B000002401E0022C06D02046FEF799FF641CDC
:10E8C000042CF7D310BD0324F6E7BDE81040FEF793
:10E8D000AFBF0000B02D002003480179C90702D066
:10E8E0000078FFF7CFB87047B02D0020F7210180E6
:10E8F0001721418000210171417170472DE9FF41CD
:10E900000026244800F0A0F92248001F074600F026
:10E910009BF9214C2149A06800900D6800E0009807
:10E920006946284004EB80000C30FFF771FF002897
:10E93000F5D101AA009901EA050304EB8303491C00
:10E94000DB6842F82030401C00910228F2D3019885
:10E9500000F0030001280BD0022810D101980321F8
:10E9600001EB90500099BDF80A6001EB900005E0C2
:10E970000198BDF80A60C0F383100844009038463F
:10E9800000F05FF908B10098A06004B03046BDE81F
:10E99000F0810000883B002070370020742E00209A
:10E9A0008AB04FF48041002001F0B0F908B1FEF7C1
:10E9B0000FF900F0FFFFFEF751F908B1FEF708F973
:10E9C000182236496846FDF751FD3548069035490D
:10E9D0004FF48070CDE9070109900723324A06A958
:10E9E0006846FEF7A1F908B1FEF7F2F82F490120B9
:10E9F000FEF7FEFF08B1FEF7EBF869460020FEF7D0
:10EA00003BFF08B1FEF7E4F82A4C2948CDE90004A1
:10EA100000256846FEF768FB08B1FEF7D9F801F05B
:10EA20007FFA08B1FEF7D4F801F0F2FC08B1FEF766
:10EA3000CFF869460120009501F08CFB08B1FEF784
:10EA4000C7F8684601F01CFC08B1FEF7C1F8FFF7F3
:10EA5000C1FD194800901948CDE9010469461848DC
:10EA6000FEF7D2FC08B1FEF7B3F802F095FF15A04F
:10EA7000FDF7C0FF1C481D49401AC008032101EBE7
:10EA800000401BA101F0C0F802F0B2FF00F0A0FFAF
:10EA90000028FBD101F058FAF8E70000C423020077
:10EAA000C42F0020C43000206D1E02006DD901006B
:10EAB000BDDE0100842D002021D30100E50D020000
:10EAC000C4310020424C4520554152542063656EAC
:10EAD0007472616C206578616D706C65207374610F
:10EAE000727465642E0D0A00B43002003C300200DE
:10EAF000424C4520554152542063656E7472616CDE
:10EB0000206578616D706C652073746172746564E2
:10EB10002E0000002DE9F047C5881E1DB6FBF5F755
:10EB20008946B6FBF5F1044605FB176C407916687B
:10EB30006843DDF820A0F718001F874200D9C61AE5
:10EB4000166001E02468491E0029FBD1A5EB0C07E3
:10EB50008846B74216D818E004EB0C00001D09EBFC
:10EB60000803BAF1000F3A4602D00146184600E009
:10EB70001946FDF77BFC2468F61B4FF0000CB844E7
:10EB8000B54201D9374600E02F46002EE4D1BDE85A
:10EB9000F087000030B5024651B101F0CBF80021FA
:10EBA000074C08E034F821301568AB4202D11160FF
:10EBB000002030BD491C8142F4D3052030BD000047
:10EBC0000000000010B531B1B2FBF3F403FB1424D4
:10EBD0001CB1092010BD0E2010BD01600021416054
:10EBE00081608281C381084610BD70B50C46054620
:10EBF000FDF710FB002802D021882868084470BD6A
:10EC000010B50A8849888A4203D1FDF745FB0120E7
:10EC100010BD002010BD70B50C460546FDF71FFB6A
:10EC2000002802D061882868084470BD10B50A88A1
:10EC300049888A4203D1FDF709FB012010BD00205D
:10EC400010BD002100F009B8012100F010B808B58E
:10EC50006A46FDF776FB009808BD08B56A46FDF7E1
:10EC600056FB08BD08B56A46FDF738FB08BD08B578
:10EC70006A46FDF73FFB009808BD08B56A46FDF7F8
:10EC80006DFB009808BD38B5044600258DF800508E
:10EC90006846FEF7C5F821686268086890420ED998
:10ECA000401E08600178238AE26801FB0325227A6E
:10ECB0002168101AC0B20A79824200D208719DF808
:10ECC0000000FEF7D1F8284638BD38B505460020CB
:10ECD0008DF800000C466846FEF7A2F8E868298A1D
:10ECE000201AB0FBF1F12A681068431C1360017010
:10ECF0009DF80000FEF7B8F838BD10B530B1017AC4
:10ED000042680368891AC9B21A6006E00E2010BD75
:10ED100003681A68541C1C601170491EC9B2F7D2EE
:10ED2000006800210171084610BDC20800F0070309
:10ED30000120895C98400840704728B1A1F1170272
:10ED4000E12A03D3072070470E207047418000203E
:10ED5000704710B560B10161F72120F8021B20F85F
:10ED6000021BFB2100F8021BFFF7C0FD002010BDB5
:10ED70000E2010BD7CB585880C46002D33D101884E
:10ED80000026102906D0112909D03A290BD055297F
:10ED90002ED129E00146204602F0C2F828E0A01D4D
:10EDA000FFF7A4FD24E02246408934F8061F814283
:10EDB00000D808466080172800D2172060801069AC
:10EDC00078B1607968B11849D1E90001CDE9000155
:10EDD000ADF802506088ADF804001369694610462A
:10EDE0009847667126717CBD0146204602F04AF9BB
:10EDF000A07A0028F7D0E1882846A5DF012580B158
:10EE00001128F0D001F0E2FB02460848084902B0A0
:10EE1000401AC00805EB0040BDE8704005A100F0B5
:10EE2000F7BEA672E5727CBD8C240200443002005D
:10EE30003C30020073645F626C655F676174746389
:10EE40005F65786368616E67655F6D74755F726535
:10EE5000717565737428292072657475726E6564A6
:10EE60002025732E000000002DE9F0410F4604001C
:10EE70004FF000050DD002F09FFB39462046FFF70A
:10EE80000DF8218881421ED1002005464FF6FF76FD
:10EE900009E00E20BDE8F081626832F81020B2422D
:10EEA00006D1401C80B28142F6D8206901F016F8E4
:10EEB000002021880BE0626832F81020B24204D1B1
:10EEC000616821F810702846E4E7401C80B2814256
:10EED000F1D80420DEE700002DE9F04791460D4609
:10EEE00004004FF0000742D0EDB302F065FB494645
:10EEF0002046FEF7D3FF2978062902D221888142D5
:10EF000002D10720BDE8F087A16800EB800601EB85
:10EF1000860001F088F830B14946284602F0B8FB77
:10EF200008B13846EEE72978DFF8488058F8212004
:10EF30002AB12069B8B1294690470028E2D1A068DB
:10EF4000294600EB860001F08DF8070006D02978ED
:10EF500058F8210010B1686800F0A3FFA068494686
:10EF600000EB860000E002E002F08EFAD9E70E2006
:10EF7000C8E700009C240200F8B505000C4620D02C
:10EF8000002C1ED02888112806D0A0F130011F299E
:10EF900002D950381F2814D8AE8820463146FEF7D3
:10EFA0007DFFADF80000218881420AD0298811290F
:10EFB00008D0A16800EB800001EB8000314602F030
:10EFC00063FAF8BD62684FF6FF7122F810106946C7
:10EFD000E06801F047F8F8BD2DE9F041044600F182
:10EFE000140700F10A05867C007A86B001F1020858
:10EFF000002814D08ADF14216846FDF750FA334602
:10F000002A46394640468BDF05218DF800100190D5
:10F01000002804D0A16A002901D06846884706B0BC
:10F02000BDE8F0814FF4C8710182062141811821A9
:10F0300081810021C1817047017D074A82615210A0
:10F04000C26121F018010022028441F0040101751F
:10F050000121417570470000A0860100F0B520B184
:10F060001AB1032903D00720F0BD0E20F0BD0479AA
:10F070000346051D0CB10420F0BD0021168808468A
:10F0800033F82170B742F7D0491C11F0FF01F7D0D7
:10F0900003EB8401641C2C7012680A60F0BD18B187
:10F0A00000214171084670470E20704710B50B468D
:10F0B000040002D0980702D009E00E2010BD5807C6
:10F0C00005D4D80603D4180701D4072010BD204664
:10F0D000FFF7E5FF580701D501206071A2710020FC
:10F0E00010BD70B50D46040010D000262660666085
:10F0F000A262EDB128792072287BA074296839B109
:10F10000142204F11400FDF7B1F904E00E2070BDE3
:10F110002046FFF791FFA86830B10168C4F80A10D3
:10F120004068C4F80E0009E02046FFF77BFF05E0C9
:10F13000FFF782FF2046FFF775FF267204F12C00CF
:10F14000E0641F20A4F85000002070BD2DE9F04FAE
:10F15000044689B000208846074606901421684678
:10F16000FDF79DF904F1140004902046FFF790FB91
:10F17000010004F14C00059011D002208DF8000030
:10F18000CDF80480A16A684688470020059989DF88
:10F1900041462046FFF720FF09B0BDE8F08FA07977
:10F1A000002107916179834621B3012106918246AE
:10F1B00094F804900026B8F81C003546089012E038
:10F1C00004EB8502D8F818000899FDF712FF28B162
:10F1D000761CF6B2BAF1000F0DD002E0BAF1000FC2
:10F1E00006D16D1CEDB24D45EAD3BAF1000F02D045
:10F1F0004E4501D009E046B19DF8080040F00400FA
:10F200008DF8080001207F1C0790CDF80480BBF129
:10F21000000F02D00698874203D0079830EA0B000F
:10F2200007D000208DF8000041462046FFF7D4FEAD
:10F2300002E003208DF80000A16A09B16846884702
:10F240000020059989DFA7E770B50D46014601F159
:10F2500008020C1D28460988143586B010291ED0D6
:10F260001B2907D01D292DD106B01146BDE87040DD
:10F27000FFF76CBF064614216846241DFDF70FF901
:10F28000207801281ED1B06A00281BD004208DF8F8
:10F290000000049520788DF80400B16A10E006465D
:10F2A00014216846FDF7FBF806208DF80000201DAC
:10F2B00001902088ADF808000495B16A002901D0BA
:10F2C0006846884706B070BD30B585B0040025D0CB
:10F2D00014216846FDF7E3F88ADF2046FFF7D8FAE5
:10F2E000012528B1A16A19B18DF8005068468847F8
:10F2F00004F14C0104F1140089DF044608280FD002
:10F3000074B1084808492246401AC00805EB00407D
:10F3100006A100F07DFC204605B030BD0E20FBE7C5
:10F320000020F9E7543002003C30020073645F6251
:10F330006C655F6761705F7363616E5F7374617248
:10F34000742072657475726E65642030782578005B
:10F3500000F180400068002800D00120704708B507
:10F3600000F18040002101600068009008BD0000AD
:10F3700070B50D4C0125207808B185260EE00020DF
:10F38000A06060602061E060084801F063F9064613
:10F3900001F08AF808B901F047F9257001F03CF94D
:10F3A00000B1A570304670BD4834002069DE010010
:10F3B00038B500258DF800506846FDF731FD084C42
:10F3C000E068401EE060E06828B901F025F910B956
:10F3D00001F04EF9A5709DF80000FDF745FD38BD20
:10F3E00048340020F0B505460478154889B0164623
:10F3F00040F82420124A0869121DA2F1080742F8B9
:10F400002400487F385520226846FDF72FF80494E1
:10F410002878385C48B10EB10A4A00E000226946FB
:10F42000281D01F0C3FB09B0F0BD0EB1064A00E093
:10F430000022694605F10C0001F06CFAF3E70000C8
:10F44000DC2D002059210200FD1F020030B403789A
:10F45000054CE35C1BB130BC001D01F0DDBB30BCD2
:10F460000C3001F0C1BA0000D82D002030B4037870
:10F47000054CE35C1BB130BC001D01F04FBC30BC3F
:10F480000C3001F027BB0000D82D00200FB408B5C8
:10F490000399002904D004AA00926A4600F00FF8EC
:10F4A00001B05DF814FB10B582680446002A05D04F
:10F4B000D4E90403216898470020A06010BD2DE91D
:10F4C000FC4791460C00804676D014F8011B39B1F8
:10F4D00025290ED04046FEF707FC20780028F4D1FD
:10F4E00098F80C00002867D04046BDE8FC47FFF7BD
:10F4F000DABF0020012221782B291BD02D2902D030
:10F50000302908D102E040F0010001E040F00200A3
:10F51000641C002AEFD100252A290ED02178A1F100
:10F5200030020A2A11D205EB850201EB4205641C68
:10F53000303DF1E740F00400EAE7D9F800100B1D78
:10F54000C9F800300968641C0D44217800232E2975
:10F550000BD114F8011FA1F130020A2A05D203EBE6
:10F56000830201EB4203303BF3E76C290DD068299D
:10F570000BD0692921D00BDC252918D0582931D08E
:10F5800063290ED0642915D117E014F8011FECE7A8
:10F59000702969D0732932D075291BD0782909D1F7
:10F5A00020E0D9F80000011DC9F80010017840469C
:10F5B000FEF79AFB641C90E76CE0D9F800100A1D76
:10F5C000C9F800200968CDE900500A224046FFF73B
:10F5D00087F8EFE7D9F800100A1DC9F8002009687C
:10F5E0000A2206E0D9F800100A1DC9F800200968AF
:10F5F0001022CDE90050404602F050FEDAE7D9F87B
:10F60000001000270A1DC9F800200E68C00705D1A8
:10F6100012E04046761C7F1CFEF766FB317800291D
:10F62000F7D104E0202140466D1EFEF75DFBBD4290
:10F63000C0D9002DF6D1BDE74EB13046FCF73AFFF8
:10F64000074604E0202140466D1EFEF74DFBBD42FB
:10F6500006D9002DF6D103E04046761CFEF744FBA8
:10F6600031780029F8D1A5E7D9F80000011DC9F8C3
:10F670000010056830214046FEF736FB78214046F1
:10F68000FEF732FB08200021CDE9000103461022DD
:10F690002946B0E7BDE8FC8770B541EA4201DDE9E3
:10F6A00004564FF0A04441EA830141EA052104EBEE
:10F6B000800041EA0641C0F8001770BD70B541EA0C
:10F6C0004201DDE904564FF0A04441EA830141EADA
:10F6D000052104EB800041EA0641C0F8001770BD27
:10F6E00070B541EA4201DDE904564FF0A04441EA19
:10F6F000830141EA052104EB800041EA0641C0F89C
:10F70000001770BD70B541EA4201DDE904564FF0C3
:10F71000A04441EA830141EA052104EB800041EA6B
:10F720000641C0F8001770BD1CB500220B460092C0
:10F7300011460192FFF7D4FF1CBD1CB500220B46F9
:10F74000009211460192FFF7DDFF1CBD1CB50021A0
:10F7500000910B46012201911146FFF7C1FF1CBD2C
:10F760001CB5002100910B46012201911146FFF7C3
:10F77000C9FF1CBD4FF0A04202EB8000D0F800276B
:10F7800022F44032C0F80027D0F8002742EA0141B5
:10F79000C0F800177047000038B5094B44181B68C3
:10F7A00000936B4608E000BF53F82010D1F82055B5
:10F7B00020C2C1F82055401C8442F5D838BD000055
:10F7C000C424020043094FF000014FF0010208D1A8
:10F7D0001307D3E94C13102900D14BB10649074B4D
:10F7E000194300F01F0082400A4203D001207047F5
:10F7F0000349F4E700207047FFC117700038000389
:10F800003F8E16F001224FF0A043824011B1C3F8A1
:10F8100008257047C3F80C2570470000034908B558
:10F820000844002101600068009008BD00600040AD
:10F8300002494058012800D0002070470060004075
:10F8400030B5154A01460020D2F8104423460AE09C
:10F85000DB681D79854205D1401C0A28F6DB4FF094
:10F86000FF3030BD1B68002BF2D1431CF9D0CB68B0
:10F870001871D2F8103443B1DB68CC681B68236080
:10F88000D2F81024D268116030BDC2F81014C968D3
:10F8900000220A6030BD0000703700207047FCF77E
:10F8A000F7BE704708B5034A00924023024A00F0B1
:10F8B00005F808BDCD1A0200D8350020F0B595B086
:10F8C0001C4615460F4608461A9E00F003FB1821F9
:10F8D00009A8FCF7E4FD0E96CDE90954002308229F
:10F8E00003A9384600F00BFB05980690BDF8100000
:10F8F000ADF81C00BDF81200ADF81E0000208DF818
:10F9000021000398082600F00300012802D00228F5
:10F9100018D032E003983346850AC0F3C2008DF850
:10F92000200003980FA9C0F38314A200384600F00A
:10F93000E6FA09A8009006AB22460FA9284600F077
:10F9400025FA1AE00398840DC0F3C2008DF8200058
:10F95000082C01D2254600E0082533462A460FA987
:10F96000384600F0CCFA2E44641B09AB06AA29469F
:10F970000FA800F073F9002CEAD1384600F0B0FA75
:10F9800015B0F0BD0A4A012902EBC00007D00229D8
:10F9900007D0032907D0042907D000207047022090
:10F9A0007047042070470079704740797047000025
:10F9B0003C30020010B5FFF772FF04210348FFF747
:10F9C0003FFF02490120C968487110BD2C30020078
:10F9D0002DE9F04F8DB0FEF79FF918B100200DB062
:10F9E000BDE8F08F7E4C4FF0000BC4F818B4BFF3A5
:10F9F0004F8F7C49A06802900D68D846284004EBE0
:10FA000080000BE0D4F8180470B961680298814254
:10FA100001D8A160E2E7284004EB80000C3002A985
:10FA2000FEF7F6FE0028EDD1002005AA029901EAB2
:10FA3000050304EB8303491CDB6842F82030401CBB
:10FA400002910228F2D3059800F00300022802D0A8
:10FA500001284DD0AAE005985022810D8946B2EBCD
:10FA6000905F00D850210E4666F39F5005900831F4
:10FA70005D4800F0E6F9070078D000F02BFA434625
:10FA8000082205A9384600F042FA029908F1080A4E
:10FA90002940681A8000001D864222D9504D0C353D
:10FAA00030B1C2B204EB8101301A90460C3104E04F
:10FAB0002946F2B2002590462846C6B2534638463B
:10FAC00000F025FA0AEB080325B1324629463846EC
:10FAD00000F01DFA029909F1030001EB9000029079
:10FAE0003BE004EB81015346324638460C31EFE7E8
:10FAF0000598C0F38310062800D30620059960F30B
:10FB00008911C1F38310801C05918100364800F0F3
:10FB100098F907004AD000F0DDF94346082205A90C
:10FB2000384600F0F4F908F1080800260FE00298C2
:10FB3000434600EA0501401C04EB810102900422C7
:10FB400038460C3100F0E3F908F10408761C0598FA
:10FB5000C0F38310B042EAD847B1D4F81054D4F8B7
:10FB6000180478B1384600F0BBF934E01EE0E868CC
:10FB70004079012804D12A682846394612689047FE
:10FB8000E8680568002DF2D1384600F0A9F98DF833
:10FB900000B06846FDF744F9D4F8180408B9029893
:10FBA000A0609DF80000FDF75FF914E0D4F8104460
:10FBB00005E02168204689688847E0680468002CD1
:10FBC000F7D10A480A49401AC008022101EB004057
:10FBD00008A100F019F8FEF79FF880F00100FEE69A
:10FBE00070370020742E0020E8300200B43002008C
:10FBF0003C3002004261636B656E647320666C7515
:10FC0000736865640000000000231A4602F02AB8F9
:10FC100008B5012300926A4602F024F808BD1CB51D
:10FC2000CDE9002302236A4602F01CF81CBD3EB554
:10FC3000069C8DE81C0003236A4602F013F83EBDC3
:10FC4000F0B587B00DF1300C9CE8F0008DE8FC00B9
:10FC500006236A4602F006F807B0F0BD2DE9F0472A
:10FC60000E4680461C469246082940D894F80C90CF
:10FC7000002020731946104601F0AEFB0025B54266
:10FC800006D218F805201BA12046FFF7FFFB03E072
:10FC90001AA12046FFF7FAFB6D1C082DEFD318A11F
:10FCA0002046FFF7F3FB0025B54212D218F8057085
:10FCB0007E2F08D8FCF7D6FB0068C05D10F03E0F21
:10FCC00001D03A4600E02E220EA12046FFF7DEFBCF
:10FCD00003E00DA12046FFF7D9FB6D1C082DE3D3EF
:10FCE00001222146504601F059FB84F80C90BDE8F2
:10FCF000F08700002025303278000000202020000E
:10FD00007C0000002563000020000000064910B5BB
:10FD100000200870054800F0E1F8002803D10448ED
:10FD200000F0F9F9002010BD70370020E830020023
:10FD3000A826020002480349401AC0087047000084
:10FD4000D43002003C30020013B56846FEF722FFB3
:10FD500008B100201CBD0248009950F831001CBDBC
:10FD60003C30020070B508480125D0F810440570F9
:10FD700007E0E06845712168204649688847E068E7
:10FD80000468002CF5D170BD703700202DE9FF47C5
:10FD900081460C9D00200C462F7B28739846164602
:10FDA0002946184601F018FB072E42D2DFE806F07C
:10FDB00004090F161F2A360049462846FFF766FB3E
:10FDC00037E0494628462268FFF760FB31E0D4E976
:10FDD000002349462846FFF759FB2AE0A068009017
:10FDE000D4E9002349462846FFF750FB21E0D4E937
:10FDF0000201CDE90001D4E9002349462846FFF776
:10FE000045FB16E004F1080007C88DE80700D4E9B7
:10FE1000002349462846FFF739FB0AE004F10800B1
:10FE20000FC88DE80F00D4E9002349462846FFF7A4
:10FE30002DFB00222946404601F0B0FA2F73BDE8A1
:10FE4000FF872DE9F041058A80462D1F4819C01C07
:10FE5000B0FBF5F0C6B24046FEF715FF041E19D000
:10FE60000020207101206071E58000272546761E64
:10FE7000C4F800800BE04046FEF705FF60B16179F1
:10FE8000491C6171286005467F1CC0F80080B7429C
:10FE9000F1D32046BDE8F081204600F002F80020B2
:10FEA000F8E72DE9F041457901466B1E002201E09B
:10FEB0000968521C9A42FBD30F680146002605E0F0
:10FEC00038460C68FEF701FF2146761CAE42F7D398
:10FED000BDE8F0810121001DFEF7B9BEFEF70DBFA0
:10FEE00010B504460121001DFEF7C7FE10F0FF0FFC
:10FEF00004D12046BDE81040FFF7D3BF10BD1CB5AC
:10FF000001920122009201AAFEF704FE1CBD1CB55D
:10FF100001920022009201AAFEF7FCFD1CBD000028
:10FF2000064910B500204870091D0860BFF35F8FB7
:10FF30000349044800F0DCFA002010BD5C2E0020CC
:10FF400040250200CC35002010B500F0ADFA08B114
:10FF500041DF10BD20BF40BF20BF10BD70B50446BB
:10FF60000C480121FEF77EFEBFF35F8F00250028BD
:10FF700009D10120074E042C08D0311F4A781AB14C
:10FF8000BFF35F8F356070BD0C70487001F0D6FD17
:10FF9000F6E70000602E00202DE9F8430446002714
:10FFA00090460E468DF800706846FCF739FF2046F3
:10FFB00000F039F838B105279DF80000FCF754FF30
:10FFC0003846BDE8F88320680568B8F1000F05D110
:10FFD0000168204600F03FF821680860E268012AC5
:10FFE0000CD0022A0ED0042A11D06068082A13D03F
:10FFF00005FB02013046FCF739FADDE76068405D39
:020000040002F8
:100000003070D9E7606830F815003080D4E7606858
:1000100050F825003060CFE700EBC501D1E90001C1
:10002000C6E90001C8E7016808684968884201D14B
:10003000012070470020704701680A68496880689D
:10004000884201D9491C00E00021914201D10120E0
:100050007047002070478068884201D9481C70476B
:10006000002070472DE9F84304464FF000080E4683
:100070008DF800806846FCF7D3FE2046FFF7DCFFD2
:1000800007000AD0207C40B14FF004089DF8000022
:10009000FCF7EAFE4046BDE8F88320684568416801
:1000A0002046FFF7D8FF2168486037B12068016813
:1000B0002046FFF7D0FF21680860E268012A14D0CB
:1000C000022A16D0042A19D0082A1CD060683146AA
:1000D00005FB0200FCF7CAF9204601F061FA21682D
:1000E0008A688242D2D28860D0E761683078485509
:1000F000F2E76168308821F81500EDE76168306843
:1001000041F82500E8E7D6E90001626802EBC50284
:10011000C2E90001E0E78268002191608268116114
:10012000826851618268D160826851608068016034
:10013000704708B5002242504058009008BD0000AA
:1001400020B1034909680160002070470E20704704
:100150002C2702002DE9FE4307460E460846FFF70E
:10016000EFFF00287AD100250095019506208DF833
:1001700000704FF00108ADF8040002958DF8028080
:100180006946202032686ADF3549364A891AC9082B
:10019000012202EB014430B100F018FA0246204679
:1001A0003149FFF735FD00958DF8008001950295E6
:1001B0008DF801806946402032686ADF30B100F076
:1001C00005FA024620462949FFF722FD00958DF8E1
:1001D0000070F720ADF802000195029569462320D2
:1001E00032686ADF30B100F0F1F90246204620495A
:1001F000FFF70EFD0095019502958DF80080694688
:10020000012032686ADF30B100F0E0F90246204692
:100210001849FFF7FDFC4FF4B0600090019502957E
:100220006946A12032686ADF30B100F0CFF902469A
:1002300020461149FFF7ECFC0095019502958DF8D9
:1002400000506946A02032686ADF30B100F0BEF984
:10025000024620460949FFF7DBFC0020BDE8FE838B
:10026000C43002003C300200602E0200A82E0200C2
:10027000F42E0200C02D02000C2E02006C2D020094
:100280002DE9F0410546076860DF804619491A48A4
:100290002A68081AC608BA4219D9022000EB064497
:1002A00016A12046FFF7B0FC20463A461FA12B6856
:1002B000FFF7B5FC4FF08050D0F80C0129688002A0
:1002C00000F10050421A204625A1FFF7A1FCB8F129
:1002D00000004FF001040AD000F078F9024604EB68
:1002E00006402AA1FFF794FC4046BDE8F0812F4864
:1002F0000470F9E7C43002003C300200496E7375A7
:100300006666696369656E742052414D20616C6C4C
:100310006F636174656420666F7220746865205332
:100320006F66744465766963652E00004368616E8C
:100330006765207468652052414D20737461727442
:10034000206C6F636174696F6E2066726F6D203010
:1003500078257820746F20307825782E00000000F2
:100360004D6178696D756D2052414D2073697A65D4
:1003700020666F72206170706C69636174696F6E62
:1003800020697320307825782E00000073645F6246
:100390006C655F656E61626C652829207265747595
:1003A000726E65642025732E00000000CB2E0020A5
:1003B00030B51548ADF5017D0078002821D04FF407
:1003C000FA7500BFADF8005280A9684661DF38B108
:1003D000052816D00DF5017DBDE83040FCF7F8BBCF
:1003E0006C460A497DA800F083F806E0D0E90021B8
:1003F000204690477DA800F092F87F980028E1D031
:10040000F4E70DF5017D30BDCB2E00203027020032
:100410007CB5194C207808B108207CBD0120A07063
:10042000002001F025FB112819D0002001F038FB35
:1004300012480026006801908DF800606846FCF7BD
:10044000EFFC0F4901A810DF05000AD00020207042
:100450009DF80000FCF708FD2DB128467CBD00206A
:100460007CBD0120F3E7A670667001F0B1FB0120AE
:1004700001F016FBF3E70000C82E0020C42602009E
:100480004DCB01000EB50749684600F031F805E094
:10049000D0E900108847684600F041F8029800282B
:1004A000F6D10EBDE026020001480078704700003A
:1004B000C82E00201FB568464BDF30B1052814D088
:1004C00004B0BDE81040FCF783BB084901A800F068
:1004D0000FF806E0D0E900210098904701A800F04D
:1004E0001EF803980028E6D0F4E71FBD4C27020051
:1004F000016009684160AFF3008010B5D0E90021C8
:100500005368994201D1002104E0D1E90034A342AB
:1005100002D01946816010BD08314160F0E7816862
:1005200000290BD0026892680A44826041684B68D7
:100530009A4203D108314160FFF7DFBF704770B5C1
:100540000D460646446804E0B2682946904718B153
:10055000246820680028F7D120682860256070BDD5
:1005600040680068704741680868002801D0026848
:100570000A60704702460020526806E08B4203D1B1
:1005800008681060012070471A461368002BF5D1E7
:10059000704700000C4A10B502F594730EE0991AEA
:1005A000C91001EBD171491002EBC1010C68844202
:1005B00001D90B4602E005D201F108029A42EED3BE
:1005C000002010BD486810BD6025020000B5FFF78F
:1005D000E1FF002800D1014800BD00004C250200C9
:1005E0004058002800D00120704708B50022425032
:1005F0004058009008BDD0F80403084000D0012006
:1006000070474058002800D00120704708B50022EC
:1006100042504058009008BD02480068002800D0B1
:10062000012070470004014008480068012110F0D3
:10063000010F06D14FF0E020C02280F80024843062
:10064000C1670349012008607047000000E100E035
:10065000180500400549024600200B790BB18520A2
:1006600070470A6001220A7170470000E42D0020E3
:10067000022010B54107C1F808034FF48270FEF75D
:100680006EFE05490120086004480168C1F300417D
:100690000029FAD110BD00000C00004018040040F1
:1006A000002802D001498001084770471125020047
:1006B0002DE9F0410E46054600F0F6FD00282846DB
:1006C00019D0FDF77FFB083800F060FE032802D048
:1006D00001280ED007E04FF0A040D0F81005E84008
:1006E00010F0010F05D003212846BDE8F041FFF7C7
:1006F00041B80221F8E700F0E3FD002822D02846A7
:10070000FDF760FB04464FF4807000EB84000E4F51
:1007100081B207EB8400D0F8102542F00102C0F846
:1007200010250846FFF77AF8002E0BD02846FDF773
:1007300049FB064951F82000002803D00120A040C1
:10074000C7F80403BDE8F081006000405C3400207D
:100750002DE9FC41DFF8B880044608EB04000027CF
:1007600090F930001346C0170E46401C01D00827F0
:100770004AE0B0781946C0F340022046FDF7FEFA81
:100780000546401C3FD0B078410717D4C0070AD0B7
:100790004FF0A04000EB8400D0F8001721F00201D8
:1007A000C0F8001707E000217378204600910A4640
:1007B0000191FEF783FF204600F068FDB0788007C6
:1007C00018D51448317800EB8500D0F81025124B6D
:1007D0001A40C0F810254FF4F8524FF4403302EAA3
:1007E000042203EA01410A43D0F810150A43C0F875
:1007F000102509E008EB0500327810F8481F41EA9F
:100800008211017000E004273846BDE8FC81000039
:100810005C34002000600040FFE0FCFF4FF0A0418E
:10082000D1F81015C14011F0010000D0012070472F
:1008300070B5194D95F8580008B1082070BD002416
:10084000661E2046FEF7BEFF10B1281980F8306002
:10085000641CE4B2202CF4D300242046FDF780FA77
:10086000641CE4B20C2CF8D300200D4968650B4CD5
:10087000C02081F8000401264020891FC1F8000132
:100880004FF4BE70FEF7CAFFA004C4F8040385F855
:100890005860002070BD00005C3400200060004003
:1008A00006E000E0034890F85800002800D001203E
:1008B000704700005C3400200121B1EB507F01D172
:1008C000012070470020704738B50D4600F0D0FD7C
:1008D000040014D000208DF800006846FCF7A0FA50
:1008E000207928B19DF80000FCF7BEFA112038BD30
:1008F0000120256020719DF80000FCF7B5FA00206A
:1009000038BD00000149024801F090BBB834002016
:10091000002000402DE9F0410546007916460F46BB
:1009200000EB40012D4A01EBC00102EB810494F879
:100930002A1011B10820BDE8F081294951F8201092
:100940002868FFF7C1FF08B11120F4E739462846AF
:10095000FCF7A4FA66603869206030004FF00106A9
:100960002FD03F7F4FF48E712868FFF73EFE4FF483
:10097000A2712868FFF739FE28681A49C0F80413E5
:1009800028684FEA471140F30730002804DB00F1E4
:10099000E02080F8001405E000F00F0000F1E020F6
:1009A00080F8141D286840F30730002809DB00F0A8
:1009B0001F0106FA01F14009800000F1E020C0F8B3
:1009C000001128680421C0F800150020A061E06132
:1009D00084F8290044F8140FA675ACE7B834002059
:1009E000C8240200800002002DE9F05F054600796E
:1009F0004FF4017600EB400303EBC000344B03EBF4
:100A000080040020636813B12B68C3F80863A369EE
:100A10004FF000096BB1E06938B1606810B1286827
:100A2000C0F804631120BDE8F09FE261012021615C
:100A300005E0C4F82490A261E160C4F81C9094F829
:100A40002910014302D1284600F045FF60680028C4
:100A5000286803D0C0F804630020E4E74FF4A276CE
:100A60003146FFF7C2FDB2464FF4927B59462868E3
:100A7000FFF7B6FD06464FF484712868FFF7B0FD16
:100A8000804651462868FFF7ABFD074648EA070055
:100A90003043EBD056EA070007D12146286800F022
:100AA000EBFEA169606A8142E0D8C4F818900EB1EB
:100AB0000320B8E70FB10F20B5E794F82910012003
:100AC0000029296801D00860C6E74860C4E7000033
:100AD000B83400202DE9F05F054600790B4600EBA5
:100AE000400101EBC000244901EB8004284600F0DE
:100AF00045F810B11120BDE8F09F62614FF0000988
:100B0000C4F82090A36084F828904FF48E784E4665
:100B100041462868FFF769FD28684FF0010AC0F8D0
:100B200008A02146286801F077F9606808BBD5F86D
:100B300000B067690FE000BF94F8280008B10F26E5
:100B400015E041465846FFF74BFD0028F4D02146FA
:100B5000584601F061F9206AB842F2D3574641463F
:100B60002868FFF73DFD0028F9D02868C760C4F861
:100B700014903046BFE70000B8340020007900EB45
:100B8000400101EBC000044901EB800040690028EE
:100B900000D0012070470000B8340020014902480D
:100BA00001F0F2BAE4340020002000402DE9F041C9
:100BB0000546164600790F46154A00EBC00102EBC8
:100BC000810494F8201011B10820BDE8F08111498A
:100BD00051F820102868FFF777FE08B11120F4E7DC
:100BE00039462846FCF79EF96660386920601EB1D8
:100BF000397F2846FDF7C8FD28680821C0F8001590
:100C00000020A061E0616061012184F82010DCE730
:100C1000E4340020CC2402002DE9F05F0446007982
:100C20000E4600EBC001DFF8F0A017460AEB810585
:100C30003046FFF741FEB0B168684FF000084FF44E
:100C4000047910B12168C1F80893A8694FF0000B2E
:100C500080B1E86948B1686810B12068C0F80493B1
:100C60001120BDE8F09F1020FBE7EF614FF0010875
:100C70002E6102E0EE60C5E9067B00254FF4887125
:100C80002068FFF7C3FC4FF4A2712068FFF7BEFC99
:100C90002068C0F83465C0F838752068B8F1000FD6
:100CA00012D0D0F8001241F02001C0F800122079D3
:100CB000D04600EBC0010AEB8100406838B12068E3
:100CC000C0F804932846CCE701210160EFE74FF418
:100CD000887A4FF4A27951462068FFF792FC0746C4
:100CE00049462068FFF78DFC06464FF49271206854
:100CF000FFF787FC014647EA06000843EBD022795C
:100D000002EBC20308EB8302C2F818B001B103255D
:100D1000002ED7D00F25D5E7E43400202DE9F04789
:100D200004460E460079274900EBC00001EB800520
:100D300017463046FFF7C0FD30B1204600F044F8BA
:100D400020B11120BDE8F0871020FBE76F61AE6095
:100D50004FF490774FF0000839462068FFF756FCB3
:100D60004FF4AC7631462068FFF750FC2068AA6843
:100D70006969C0F84425C0F8481520684FF001099A
:100D8000C0F808906868D0B9BA4651462068FFF7A5
:100D900038FC074631462068FFF733FC0743F4D0A0
:100DA00010B14FF00F0808E02068C0F80C903146F1
:100DB0002068FFF726FC0028F9D000206861404633
:100DC000C0E70000E43400200079054900EBC000D2
:100DD00001EB80004069002800D00120704700002E
:100DE000E4340020FBF7F4BE2DE9F84F05460C462D
:100DF0000888B5F8CA12884279D195F8C6024FF032
:100E0000000A00EB8001C1EB801005EB4006608812
:100E1000002860D13079E288A71D8146D1B250FA0E
:100E200082F2062A02D80844307111E0062030719F
:100E3000374838493288401AC108022000EB014087
:100E400080463549FEF7E4FE40463449FEF7DCFEB5
:100E500048460022D0461BE000EBC00102EB8203B3
:100E600007EB430306EB4101D3F802C0C1F80AC007
:100E7000D3F806C0C1F80EC05B894B82A1F814807C
:100E8000A1F81680A1F81880401CA1F81A80521C05
:100E900031798142E0D895F8C61200EBC00001EB31
:100EA0008102C2EB811105EB410136F8100009897E
:100EB000884210D2307906280DD085F8C5022188E5
:100EC0002846FCF787FF002811D022882946BDE874
:100ED000F84FFDF7EBB885F8C5A222886946284689
:100EE000FCF7F2FF28B122882946FDF7DFF8BDE8BC
:100EF000F88F9DF800000028F9D0228801212846AB
:100F0000FDF77AF82188284600F072F9EFE7000033
:100F10003C3002003C300200E0270200282802009A
:100F200070B502468888C97B02EBC004A41D022963
:100F300001D15188218021886288914213D9A5DF8F
:100F4000012578B111280FD0FFF740FB0246074872
:100F50000749401AC00805EB0040BDE8704005A1F4
:100F6000FEF756BE657170BD257170BD443002003C
:100F70003C30020073645F626C655F676174746328
:100F80005F65786368616E67655F6D74755F7265D4
:100F9000717565737428292072657475726E656445
:100FA0002025732E00000000F8B505460C46088881
:100FB000B5F8CA12884255D195F8C602A21D00EBB9
:100FC0008001C1EB801005EB400695F8C50200EBEF
:100FD000C00006EB400160880A3138B329E000BF49
:100FE00000EB400302EB43039F88B7F5245F0CD06E
:100FF0006FF4245C17EB0C070AD0012F02D0072FE7
:101000000BD108E05B884B8107E05B888B8104E0B3
:101010005B88CB8101E05B880B824B892BB18B898C
:101020001BB1CB890BB10B8A1BB9401C13888342BF
:10103000D6D800208DF8000095F8C5023179401C03
:10104000884203D101208DF8000010E085F8C50228
:10105000228869462846FCF737FF20B122882946B6
:10106000FDF724F8F8BD9DF800000028FAD022888A
:1010700001212846FCF7C0FF2188284600F0B8F877
:10108000F8BD00007CB506468D88C88806EBC5040F
:10109000A41D172800D217202188814200D80846B5
:1010A00060800020207121882846B5DF60B1FFF7FD
:1010B0008DFA02460F481049401AC008012101EB81
:1010C00000400EA1FEF7A4FD6079002810D1306920
:1010D00000280DD01549D1E90201CDE90001ADF894
:1010E00002506088ADF80400326969463046904786
:1010F0007CBD0000443002003C30020073645F623B
:101100006C655F67617474735F65786368616E674F
:10111000655F6D74755F7265706C792829207265E2
:101120007475726E65642025732E00008C24020095
:1011300070B505460C4690F8C602228800EB800187
:10114000C1EB801005EB4001B5F8CA02824238D1EC
:10115000608848B100212846FCF74EFF21882846C8
:10116000BDE8704000F044B8E268C1F80620E288AB
:1011700095F8C412D0B251FA82F2062A03D8084474
:1011800085F8C40211E0062085F8C4020D480E4916
:10119000401AC108022000EB01460CA13046FEF7C0
:1011A00033FD30461149FEF72FFD21882846FCF714
:1011B00011FE002805D022882946BDE87040FCF7C2
:1011C00075BF70BD3C3002003C3002004E6F742091
:1011D000656E6F75676820737061636520666F72F6
:1011E0002073657276696365732E0000842802009F
:1011F00070B588B00D46044620216846FBF74FF9CC
:1012000094F8C7021E4B401CC0B284F8C702DA68CB
:10121000002190422CD284F8C51294F8C602194ECF
:10122000401CC2B202EB820084F8C622C0EB8210DE
:1012300006EB820204EB4000126802600171022199
:101240008DF800100121ADF810100068CDF81200E3
:101250000D48CDE902042A4669469868FDF73CFE30
:10126000002803D02A462146FCF720FF08B070BDB5
:1012700084F8C81229462046FCF7A6FEF6E70000CF
:10128000C82D002030340020ADE0010010B5054924
:10129000C20800F00703885C01249C402043885466
:1012A00010BD0000B03400200449084490F930001B
:1012B000082801DB01207047002070475C340020C3
:1012C0000449084490F93000082801D201207047F1
:1012D000002070475C3400202DE9F05F2A4F06465D
:1012E0004FF0A04A4FF0010B0024381990F950102C
:1012F000491C3CD090F85000314620F0C0052846EB
:10130000FDF713FD20B3204600F040F881460AEBBC
:101310008500D0F80007C0F30148B8F1020F18D0DB
:1013200002212846FEF726FA0BFA05F1CAF8201525
:101330002846FCF747FD57F820204AB14846B9F146
:10134000030F11D0B8F1020F05D0B8F1030F07D089
:101350000DE00321E5E74846B9F1010F04D006E0AE
:101360004846B9F1020F02D1014628469047641C55
:10137000042CBAD3324601210020FEF70DFA306862
:101380000028B1D1BDE8F09F5C3400200249084438
:1013900090F85000800970475C34002010B50C466E
:1013A000017A052908D0407A38B1084808A10268B6
:1013B0002046FEF76BF800E01AB106A12046FEF7C2
:1013C00065F82046BDE81040FEF76DB8A42E002059
:1013D000257300000D0A000038B5C3880D46044689
:1013E00033B114A0009015A216A12846FEF74EF8BE
:1013F000217A05291CD0607A48B1A088FEF7C2FA8C
:10140000164951F8202016A12846FEF73FF8A0887B
:101410000021FEF799FC03461049207A143951F84F
:10142000202001B02846BDE830400EA1FEF72EB8BE
:1014300038BD00001B5B306D000000001B5B313BC2
:1014400033316D0025734C6F67732064726F707059
:101450006564202825642925730D0A00A42E002028
:10146000257300003C25733E2025733A20000000C0
:101470000349884201D103487047002070470000AB
:1014800000200040EC2D0020F0B591B00E4607463C
:1014900001226946FEF780FD04005AD19DF8000044
:1014A00004AD06285DD2DFE800F0030A181F2327E9
:1014B000BDF81220BDF810103046A1DF0BE00CA8DB
:1014C00006900146BDF8162000230198FEF717FD8F
:1014D00029463046A3DF044626E0BDF8101030460A
:1014E0000DF112029BDFF6E7294630469DDFF2E759
:1014F000294630469EDFEEE70CA807900023022223
:1015000008A90198FEF7FBFC08A80690BDF820206A
:10151000022307990198FEF7F2FCBDF820E0294666
:101520003046AEDF040016D0112C12D09DF800001A
:10153000114951F8200010B10198FEF7B2FC0022C9
:1015400069463846FEF728FD22463146684600F0D7
:101550007BF811B0F0BDBDF820008645E6D00C2424
:10156000E4E706480649401AC008022101EB0040A2
:1015700004A1FEF749FBD9E79C2402004C3002008D
:101580003C300200556E696D706C656D656E7465FA
:10159000642047415454205265717565737400008E
:1015A00001680A684968914201D3881A70478068C7
:1015B000801A0844401C704770B58CB00446C0685F
:1015C000002209A9FEF7E8FC104D1BE0BDF824102D
:1015D000A06801EB810100EB810607E09DF80000A7
:1015E00055F8200010B10198FEF75BFC0022694617
:1015F0003046FEF7D1FC0028F0D0002209A9E068AF
:10160000FEF7CAFC0028E1D00CB070BD9C2402009B
:1016100070B50C4B00210A4ADC680DE002EB810535
:101620008678AD78B54206D132F821500688B542A9
:1016300001D1586870BD491CA142EFD3002070BD94
:1016400030340020C82D0020F8B515000E460446A1
:1016500016D00C480C490095401AC008012101EB36
:101660000040227833460949FEF7E1FAA368002BCF
:1016700006D0E16801B032462846BDE8F040184780
:10168000F8BD00004C3002003C300200CC280200C3
:101690002DE9F041044600780E46002504F11001C2
:1016A000062828D2DFE800F003080B111418628A1C
:1016B000218A3046A1DF0DE03046A3DF0AE0218A0F
:1016C00004F1120230469BDF04E030469DDF01E06A
:1016D00030469EDF054605E0A06907883046AEDF4C
:1016E000050002D0112D18D00FE0A0690088B84283
:1016F0000BD00C2509E00A480A49401AC00802210B
:1017000001EB004008A1FEF77FFA2A463146204649
:10171000FFF79AFF0120BDE8F0810020FBE7000001
:101720004C3002003C300200556E696D706C656D86
:10173000656E746564204741545420526571756527
:101740007374000070B50546FCF7DDFD134C40B125
:10175000D4E904024FF08071411842F10000C4E95D
:10176000041000212846FCF71BFD30B1606820B151
:10177000606800F0C1FA0020606001212846FCF793
:101780000FFD18B1FCF774FFC4E90601284600F00C
:10179000DFFA2846BDE8704000F034B8102E002073
:1017A00070B5054600200C460870FCF761FFD5E9CE
:1017B0000223101A63EB010300263146361A9941C1
:1017C00012DAB0F5350F03D3FBF736FA0B4942189E
:1017D0004FF4960300210A48FCF7A1FD10B10D2833
:1017E00006D009E0012070BD00210548FCF7CEFCC1
:1017F000284600F081FA2070002070BDFFFFB40081
:10180000182E0020F8B51A4C074600261948FEF796
:10181000A7FED0B1616871B1D0E902106268D2E967
:101820000232C91A904120D26068007F18B1616805
:101830001048FEF784FE00F0F7F905466946FFF709
:10184000AFFF98B1606840B10AE0606800280CD131
:101850003846BDE8F840FCF75EBD3846FCF757FD5A
:1018600065609DF800000028D0D1F8BD6660CDE726
:10187000102E0020E024020070B5054688690C4651
:1018800000284FF4847128460AD0FEF7AEFED5F842
:101890001805626AE1688854606A401C606270BD25
:1018A000FEF7A3FED5F8180570BD1FB501238DF80E
:1018B0000030CDE90121D0E90012684690471FBDF4
:1018C0001FB501238DF80030CDE90121D0E90012C8
:1018D000684690471FBD10B5044600684FF49271EA
:1018E000FEF783FE4FF484712068FEF77EFE2068C9
:1018F0000121016010BD00007FB501460378144846
:10190000144A801AC008032202EB0040042B18D0AE
:10191000052B0ED0062B0BD14968CA788D794C79EE
:101920000B798DE83C008B784A780BA1FEF788F99B
:101930007FBD48680028FBD004B0BDE87040FBF7CD
:1019400047B911A1FEF760F9BDE87F4000F050B83B
:10195000B43002003C300200436F6E6E6563746900
:101960006E6720746F207461726765742025303251
:10197000782530327825303278253032782530326B
:1019800078253032780000005363616E2074696DF1
:101990006564206F75742E001FB5002000900190C3
:1019A0000290039001208DF804008DF80C000D4A80
:1019B00069460D48FDF795FB08B1FBF709F90B4A9D
:1019C00003210948FDF74AFB08B1FBF701F90022A2
:1019D00004210548FDF76AFB002801D0FBF7F8F861
:1019E0001FBD0000F9180200F0310020C0230200E2
:1019F00010B50848FDF768FC08B1FBF7E9F80120CD
:101A0000FBF7EAFF002803D0BDE81040FBF7E0B881
:101A100010BD0000F031002038B50021012548B18B
:101A2000012810D003280DD1FEF7FEFDBDE8384097
:101A3000FDF7BEBC4FF0E020C0F88051BFF34F8FE0
:101A4000BFF36F8F38BD8DF800106846FBF7E8F9DB
:101A5000064C207808B9FDF78BFCE068401CE0607C
:101A6000A5709DF80000FBF7FFF938BD4834002051
:101A70003EB5044609496846FEF73AFD08E000BF56
:101A8000D0E900212046904730B16846FEF747FD77
:101A900002980028F4D13EBD11203EBDC8260200A8
:101AA0003EB5044608496846FEF722FD07E000BF40
:101AB000D0E90021204690476846FEF730FD0298A5
:101AC0000028F5D13EBD0000D42602002DE9F041EA
:101AD0001400884618D000250E4F032608EB050198
:101AE00022460020FAF7D6FD0544241A40B938787A
:101AF000002809D008494FF47A408847761E05D05F
:101B000001203870002CE9D1BDE8F0810020387048
:101B1000FAE70000682E0020A126020010B5044656
:101B20000020FBF759FF08B1FBF752F824B9FBF787
:101B3000BFFE08B1FBF74CF8012010BD70B5194D80
:101B4000194C07E0016820788847002829D01548FB
:101B5000FEF7E5FCA8680028F4D1FEF703F900BF02
:101B6000FDF736FF0028FBD1207803280CD002288F
:101B70000AD0FEF799FC00B133DF0C490120086060
:101B8000BFF34F8F20BFFDE7BFF34F8F08480168B9
:101B9000084A01F4E06111430160BFF34F8F00BFB9
:101BA000FDE770BDCC3500205C2E00200005004014
:101BB0000CED00E00400FA05002805D103490120DE
:101BC00048700020FCF73CB9704700004834002002
:101BD00010B51620FAF726FFA0B1114890F80004BE
:101BE0004009082811D20121814011F0EC0F0CD0DE
:101BF0000C4882684FF480016AB1016841F48001A9
:101C0000016010BD42F2010001E042F20200BDE8B5
:101C10001040FAF7DDBF4FF0E020C0F8001110BD12
:101C200016E000E0C03500200148FEF79CBC000033
:101C3000E0240200C207002A03D000BF4FF00F02C9
:101C400001E04FF0F00201D04FEA0111044B03EB29
:101C50005003187800EA020040EA0100187070474B
:101C6000283500202DE9F84F07462148914688463F
:101C700005681E46012269461846FBF7EBFFDFF8B0
:101C800074A060B3009800210446801C0AE000BFE5
:101C900000EA050259F821C00AEB8202401C491CE7
:101CA000C2F80CC0B142F3D34FEA1749FCF764FA0B
:101CB000611C29400AEB810149EA00422C40CA60BC
:101CC0000AEB8401C86867F3C50066F3891068F3FE
:101CD0009F2020F00300401C20F00400C8609AF808
:101CE000000001E0FDF774FE0028FBD1BDE8F88F8D
:101CF000742E00207037002070B50446124800256D
:101D00000078F8B1F4B1207FE0B1FCF7B1FCD4E980
:101D10000223801A994110D32069002600B9267742
:101D2000D4E905108847206960B1217F51B1D4E919
:101D3000022110187141C4E9020121460348FEF74F
:101D4000FEFB0125284670BD102E0020E024020075
:101D5000F8B51B4C69462068FCF75DFF002601279B
:101D6000184D29E0017821B101290CD002291BD19D
:101D700014E041680A7FBAB90F774168104808300B
:101D8000FEF7DDFB10E041686868814201D16E60BA
:101D90000AE00B480830FEF7EDFB05E0FFF744FFD3
:101DA00008B10677FAE72F7069462068FCF728FF2C
:101DB00069462068FCF72FFF0028D3D1F8BD00004A
:101DC000D8240200102E0020F8B50B4C0D46064614
:101DD00069462068FCF709FF58B1067045606946FE
:101DE0002068FCF723FF10B10448FCF779FA0020C3
:101DF000F8BD0420F8BD0000D8240200182E0020F1
:101E0000034880684108034800224068FAF754BF3D
:101E1000F82D0020D024020070B50C4605464FF482
:101E20008E71FEF7E2FB216AA068415C206A401CCB
:101E30002062C5F81C1570BD1FB500228DF800206A
:101E40000291816801914261D0E900126846904791
:101E50001FBD1FB500228DF80020029181680191FD
:101E60004261D0E90012684690471FBD70B5027804
:101E7000044662B11C481D4B0121C01AC00801EB89
:101E80000040012A27D0022A24D119A124E0264C9F
:101E9000244D60882844FAF72DFF6088401C80B2EA
:101EA0002918608011F8011C0A2904D00D2902D0DC
:101EB000218888420ED31B49628801F53D70FBF7EB
:101EC00045FB082804D01328F5D008B1FAF780FEA6
:101ED0000020608070BD15A1FDF796FE6068BDE82A
:101EE0007040FAF775BE0000B43002003C300200CA
:101EF000436F6D6D756E69636174696F6E20657295
:101F0000726F72206F63637572726564207768699F
:101F10006C652068616E646C696E6720554152542F
:101F20002E000000D02E0020B02700204572726FD6
:101F300072206F6363757272656420696E20464912
:101F4000464F206D6F64756C652075736564206203
:101F50007920554152542E007CB50178254DA1B30E
:101F600001290BD002291DD18DF80010C068691C11
:101F700001900122C81DFDF769FA30E0017A59B1DC
:101F8000406801781C48FAF749FE1B4C012650B105
:101F90008DF8006001900DE016490122491CC81D12
:101FA000FDF754FA7CBDA068E168814205D00020AD
:101FB0008DF80000696868468847A068E168081ADB
:101FC000A1888842E8D9AE707CBDFFE70A4809497C
:101FD0001030FAF708FE30B103208DF80000696870
:101FE00068468847F0E70349012201F10800FDF740
:101FF0003DFAE9E7342E0020A03500201FB50A463F
:1020000001788DF8001041680191017A8DF808106F
:10201000C0680390044850F82210001F50F8222096
:10202000684690471FBD0000E02D00202DE9FF47C6
:102030000C4605464FF40071FEF7DDFA01274FF418
:102040000178002618B34FF4927949462846FEF7E6
:10205000C7FAE0B149462846FEF7C7FAC5F8088333
:1020600094F8290000B96F6002208DF80000D5F8BF
:102070008004C5F880040390A0690290E068019094
:10208000A661E661D4E900126846904728E0042181
:102090002846FEF7B0FA18B34FF484712846FEF7CD
:1020A0009FFAE8B121462846FFF7E6FB616AA0697E
:1020B000884215D1E06938B1E268616AA06120699F
:1020C000E6616662E06008E094F8290000B96F609C
:1020D000C5F80883A661E268616A2046FFF7E5FB60
:1020E0004FF48E7841462846FEF77AFA80B160694F
:1020F000216A814202D294F8280028B3414628463A
:10210000FEF773FA606918B161692046FFF794FE23
:102110004FF4A27841462846FEF762FA002818D00C
:1021200041462846FEF761FA94F8290000B12F6075
:10213000A06900280DD0A661E268616A04B020465B
:10214000BDE8F047FFF7B1BB21462846FFF764FE24
:10215000DEE7BDE8FF8700001FB50A4601788DF86D
:10216000001041680191017A8DF80810C068039051
:10217000044850F82210001F50F82220684690476B
:102180001FBD0000E02D00202DE9FF410C464FF45B
:10219000927705463946FEF734FA0026B8B139463B
:1021A0002846FEF733FA02208DF80000D5F88004A7
:1021B000C5F880040390D5F83C050290E0680190D2
:1021C000A661E661D4E900126846904723E04FF427
:1021D000887739462846FEF714FAE0B13946284692
:1021E000FEF714FAD5F83C15A069884213D1E069CE
:1021F00060B1E268D5F8000220F02000C5F80002C6
:10220000E069A0612069E661E06001E0A661E26842
:102210002046FFF755FB4FF4A27739462846FEF7D4
:10222000F0F968B139462846FEF7F0F9A06938B1EF
:10223000A661E661D5F83C152046E268FFF740FB51
:102240004FF4907631462846FEF7DBF960B131460F
:102250002846FEF7DBF90120E860606920B1D5F877
:102260004C152046FFF7F5FD4FF4AC763146284675
:10227000FEF7C7F900280ED031462846FEF7C6F90A
:102280006069002807D0D5F84C1504B02046BDE899
:10229000F041FFF7DEBDBDE8FF8100002DE9F05FF2
:1022A0008346DDE90A4A994690460D4608460127CD
:1022B00003E000BFB0FBF8F07F1C4045FAD2B945FF
:1022C00000D94F465FEACA7012D18CB15FEA8A70BA
:1022D00002D5B9F1000F01D0202607E0302605E035
:1022E00031465846641EFBF7FFFC0CB1A742F7D3FA
:1022F0005FF00106B9F1010F02D9A9F1010903E06C
:10230000B5FBF6F0404502D306FB08F6F2E7DFF82E
:102310003C9000BFB5FBF6F000FB165519F8001015
:102320005846FBF7E1FCB6FBF8F6002EF2D15FEA67
:10233000CA7009D0002C07D0A74205D220215846E8
:10234000641EFBF7D1FCF5E7BDE8F09F16250200FF
:1023500070B50C460546FBF7EBFC002807D0426839
:10236000002A04D021462846BDE87040104770BDC1
:1023700010B5042817D209B1032400E00024FBF7AC
:10238000E5F94FF0A04101EB8000D0F8001721F4EF
:102390004031C0F80017D0F8001741EA0441C0F8F6
:1023A0000017002010BD062010BD0000E432002000
:1023B0004432002004000000200000000100000062
:1023C00001000200080000000600000005000000F7
:1023D000070000000000000000E0D7010D0E0F1004
:1023E0000B0C1819C0330020E033002010340020FB
:1023F0000B000300D1D801000C000300D1D801006C
:1024000018000300D1D8010019000300D1D8010041
:1024100001000000000000000000000000000000BB
:1024200000000000000000000000000000000000AC
:10243000000000000000000000000000000000009C
:10244000000000000000000000000000000000008C
:10245000000000000000000000000000000000007C
:10246000000000000000000000000000000000006C
:10247000000000000000000000000000000000005C
:10248000000000000000000000000000770A0000CB
:1024900000000000770A00000000000000000000BB
:1024A00005E6010000000000000000000000000040
:1024B00031E601009ECADC240EE5A9E093F3A3B542
:1024C0000000406E00000050050902009D0B020054
:1024D0000300000008350020383500200100060008
:1024E00000000000302E002085DE0100FFFFFFFF0E
:1024F000FFFFFFFFFFFFFFFFFFFFFFFF00000000E8
:10250000000000000000D6010601000000000000ED
:102510000338FDD8704730313233343536373839E7
:102520004142434445460000000000000000000016
:102530001031020014310200000000000000000011
:10254000282502004025020004000000556E6B6E35
:102550006F776E206572726F7220636F6465000022
:1025600000000000902C0200010000003C2B020043
:10257000020000003029020003000000B02B02001E
:1025800004000000042C020005000000E42A020000
:1025900006000000802A020007000000EC2B020069
:1025A00008000000F82A0200090000005C2B02006D
:1025B0000A000000782C02000B000000182902001D
:1025C0000C000000102B02000D000000E02C0200A7
:1025D0000E000000DC2B02000F000000182C02008F
:1025E000100000004C2C020011000000F42C02002E
:1025F00012000000C82C020013000000642C02002E
:1026000080000000982A020081000000D429020006
:102610008200000094290200830000007429020057
:1026200084000000B029020085000000BC2A0200DE
:1026300086000000C42B020090000000602A020007
:10264000910000005429020092000000242B020097
:10265000008200002C2C020001820000782B020076
:1026600002820000942B020000840000F029020086
:10267000018400009C2C020002840000382A020021
:1026800003840000142A0200A5F80100A3F8010049
:102690009DF80100000000000000000000000000A4
:1026A0000338FDD870470000D83600207F000000B6
:1026B000583700200000000000000000000000006B
:1026C0000000000001000007B4260200C42602003A
:1026D00008000000EC260200FC26020008000000B2
:1026E000FC2602000C2702000800000064310200F2
:1026F0006C310200000000000000000054310200B4
:102700006431020000000000000000000000000032
:1027100000000000143102003C3102003C31020094
:1027200044310200443102004C310200B027002045
:102730000C2702002C270200080000004C31020088
:102740005431020000000000000000003C2702009D
:102750004C2702000800000000404040404040403C
:102760004040414141414140404040404040404064
:102770004040404040404040400502020202020208
:102780000202020202020202022020202020202057
:10279000202020020202020202029090909090906B
:1027A0001010101010101010101010101010101029
:1027B000101010100202020202028888888888889D
:1027C0000808080808080808080808080808080889
:1027D000080808080202020240000000592702000F
:1027E0004E6F7420656E6F756768207370616365E6
:1027F00020666F72206368617261637465726973C9
:1028000074696373206173736F63696174656420B5
:1028100077697468207365727669636520307825FE
:102820003034582021000000496E63726561736581
:1028300020424C455F474154545F44425F4D4158EC
:102840005F434841525320746F2062652061626C7F
:102850006520746F2073746F7265206D6F726520D0
:10286000636861726163746572697374696373200C
:10287000666F72206561636820736572766963654F
:1028800021000000496E63726561736520424C450A
:102890005F44425F444953434F564552595F4D414F
:1028A000585F53525620746F2062652061626C65D8
:1028B00020746F2073746F7265206D6F7265207362
:1028C00065727669636573210000000053442047F8
:1028D0004154542070726F636564757265202825B9
:1028E0006429206661696C6564206F6E20636F6E79
:1028F0006E656374696F6E2068616E646C65202517
:10290000642077697468206572726F723A2030783B
:10291000253038582E0000004E52465F4552524F27
:10292000525F494E56414C49445F44415441000076
:102930004E52465F4552524F525F534F46544445A4
:10294000564943455F4E4F545F454E41424C4544C6
:10295000000000004E52465F4552524F525F4645BE
:1029600041545552455F4E4F545F454E41424C4590
:10297000440000004E52465F4552524F525F4D5543
:102980005445585F554E4C4F434B5F4641494C456B
:10299000440000004E52465F4552524F525F4D5523
:1029A0005445585F4C4F434B5F4641494C454400AA
:1029B0004E52465F4552524F525F4D555445585FF7
:1029C000434F4E445F494E49545F4641494C45444C
:1029D000000000004E52465F4552524F525F4D5527
:1029E0005445585F494E49545F4641494C4544005F
:1029F0004E52465F4552524F525F424C455F4950DE
:102A000053505F52585F504B545F5452554E4341A0
:102A1000544544004E52465F4552524F525F424C1D
:102A2000455F495053505F504545525F52454A45B6
:102A300043544544000000004E52465F4552524FF9
:102A4000525F424C455F495053505F4C494E4B5F7B
:102A5000444953434F4E4E45435445440000000003
:102A60004E52465F4552524F525F4150495F4E4F62
:102A7000545F494D504C454D454E5445440000006F
:102A80004E52465F4552524F525F4E4F545F535520
:102A900050504F52544544004E52465F4552524F9B
:102AA000525F4D4F44554C455F4E4F545F494E4920
:102AB0005449414C495A4544000000004E52465F7B
:102AC0004552524F525F4D4F44554C455F414C5219
:102AD000454144595F494E495449414C495A45443E
:102AE000000000004E52465F4552524F525F4E4F1B
:102AF000545F464F554E44004E52465F4552524F2A
:102B0000525F494E56414C49445F5354415445002D
:102B10004E52465F4552524F525F444154415F53BB
:102B2000495A45004E52465F4552524F525F494FF7
:102B30005F50454E44494E47000000004E52465FEC
:102B40004552524F525F5356435F48414E444C45A5
:102B5000525F4D495353494E470000004E52465F65
:102B60004552524F525F494E56414C49445F4C4585
:102B70004E475448000000004E52465F4552524FA7
:102B8000525F4452565F5457495F4552525F414E1F
:102B900041434B004E52465F4552524F525F4452A2
:102BA000565F5457495F4552525F444E41434B0074
:102BB0004E52465F4552524F525F494E5445524E17
:102BC000414C00004E52465F4552524F525F5354A3
:102BD0004F524147455F46554C4C00004E52465FB0
:102BE0004552524F525F4E554C4C00004E52465F7C
:102BF0004552524F525F494E56414C49445F5041F5
:102C000052414D004E52465F4552524F525F4E4F19
:102C10005F4D454D000000004E52465F4552524FF9
:102C2000525F464F5242494444454E004E52465F21
:102C30004552524F525F4452565F5457495F455276
:102C4000525F4F56455252554E0000004E52465F5D
:102C50004552524F525F494E56414C49445F4144A0
:102C6000445200004E52465F4552524F525F524509
:102C7000534F5552434553004E52465F4552524FB3
:102C8000525F494E56414C49445F464C41475300C0
:102C90004E52465F53554343455353004E52465F91
:102CA0004552524F525F424C455F495053505F432B
:102CB00048414E4E454C5F414C52454144595F4559
:102CC00058495354530000004E52465F4552524FEC
:102CD000525F434F4E4E5F434F554E54000000002D
:102CE0004E52465F4552524F525F54494D454F55E3
:102CF000540000004E52465F4552524F525F4255BB
:102D0000535900007761726E696E67006465627581
:102D1000670000001B5B313B33306D001B5B306D87
:102D2000000000001B5B313B33316D001B5B313B0E
:102D300033326D001B5B313B33336D001B5B313B2A
:102D400033346D001B5B313B33356D001B5B313B16
:102D500033366D001B5B313B33376D00696E666F38
:102D6000000000006572726F7200000073645F62A1
:102D70006C655F6366675F7365742829207265748C
:102D800075726E6564202573207768656E206174A6
:102D900074656D7074696E6720746F20736574203C
:102DA000424C455F47415454535F4346475F534548
:102DB00052564943455F4348414E4745442E000023
:102DC00073645F626C655F6366675F73657428290F
:102DD0002072657475726E6564202573207768654E
:102DE0006E20617474656D7074696E6720746F20F5
:102DF00073657420424C455F434F4D4D4F4E5F43CA
:102E000046475F56535F555549442E0073645F62D1
:102E10006C655F6366675F736574282920726574EB
:102E200075726E6564202573207768656E20617405
:102E300074656D7074696E6720746F20736574209B
:102E4000424C455F47415454535F4346475F4154AA
:102E500054525F5441425F53495A452E00000000CE
:102E600073645F626C655F6366675F73657428296E
:102E70002072657475726E656420257320776865AD
:102E80006E20617474656D7074696E6720746F2054
:102E900073657420424C455F434F4E4E5F43464737
:102EA0005F4741502E00000073645F626C655F6392
:102EB00066675F73657428292072657475726E6524
:102EC00064202573207768656E20617474656D7069
:102ED00074696E6720746F2073657420424C455F7F
:102EE0004741505F4346475F524F4C455F434F5504
:102EF0004E542E0073645F626C655F6366675F7338
:102F0000657428292072657475726E656420257356
:102F1000207768656E20617474656D7074696E6782
:102F200020746F2073657420424C455F434F4E4EB2
:102F30005F4346475F474154542E0000626C655F13
:102F400064625F64697363006E72665F626C655F82
:102F500067617474000000006E72665F626C655F8A
:102F600067710000626C655F7363616E0000000052
:102F7000626C655F6E75735F63000000636C6F6306
:102F80006B000000434C4F434B0000004750494F3B
:102F90005445000050525300554152540000000067
:102FA00055415254450000006170705F6275747441
:102FB0006F6E00006170705F74696D657200000073
:102FC0007077725F6D676D7400000000736F7274CC
:102FD0006C697374000000007274745F6C6F675FDB
:102FE0006261636B656E6400617070006E72665F33
:102FF000736468006E72665F7364685F626C65001C
:103000006E72665F7364685F736F63006C31020099
:10301000B02700202007000034C50100D431020091
:10302000D02E0020481F000014CA0100882602008C
:1030300000000000D82F02006C2E00203C2F020060
:1030400000000303482F020000000303582F020072
:1030500000000303642F020000000303702F02002E
:10306000000003037C2F020000000000842F0200F8
:10307000000000008C2F020000000000942F0200CE
:1030800000000000982F020000000000A02F0200A6
:1030900000000000A82F020000000000B42F020072
:1030A00000000000C02F020000000000CC2F020032
:1030B00000000000E82F020000000303EC2F0200D4
:1030C00000000303F42F020000000303003002009D
:1030D00000000303A82D00209E2D0020A62D002017
:1030E000FC32002018000000802E0020782E0020E6
:1030F000802E00201836002018000000F03200203A
:103100009A2D0020010000000200000001000000D4
:103110001D1B020075ED0100DC3100200DD1010006
:10312000B427002049F20100F031002079EF0100BE
:10313000842D0020B1D201000000000061D4010004
:10314000C431002091D1010000000000B91B020031
:1031500000000000B103020000000000B5040200FE
:1031600000000000191A02000000000002FF140114
:10317000FF01CF03FFFFFF01FF01FF713201139831
:103180002D1520AC230214FC30021AD404037FFF57
:10319000FF15100140110222041220BA4008011F3D
:1031A00029D7091EDB14642D021A04041A5C041AC0
:1031B0000C041A1C041A14041A24041A2C041A34B9
:1031C000041A3C041A44041A4C041A54045104000E
:0431D00090D0030098
:040000050001C20133
:00000001FF
